:100000000C943E001895000018950000189500000B
:10001000189500001895000018950000189500002C
:10002000189500001895000018950000189500001C
:100030001895000018950000189500000C940B35D9
:1000400018950000189500000C944635189500008E
:1000500018950000189500001895000018950000EC
:1000600018950000189500001895000018950000DC
:100070001895000018950000189500008FEF8DBFAF
:10008000C0E8E8E94E2E80E18EBFD0E1FFE05F2EB0
:10009000A89584B7082E877F84BF88E1992780932D
:1000A000600090936000EEEFFFE0A0E0B1E08827F1
:1000B0008D933197E9F787E68093C40080E08093C1
:1000C000C50088E18093C10066247FE371B90E9476
:1000D000593780E08093800081E08093810081E047
:1000E00085BD86E085BD80E084BD70916E007E7F19
:1000F00070936E0070916F007E7F70936F00F89424
:1001000087E880937A0080E480937C00089A099ABB
:100110000A9A0B9A0C9A0D9A0F9821982298239874
:10012000249A0E9A2098539A549A559A569A289A35
:10013000299A2A9A2B9A5E982C98169801080800FA
:1001400000000000000000000000065F0600000044
:10015000000703000703000000247E247E24000023
:1001600000242B6A1200000000631308646300007F
:100170000036495620500000000007030000000030
:1001800000003E41000000000000413E0000000071
:1001900000083E1C3E0800000008083E0808000059
:1001A0000000E060000000000008080808080000E7
:1001B0000000606000000000002010080402000041
:1001C000003E5149453E00000000427F40000000D3
:1001D0000062514949460000002249494936000061
:1001E000001814127F100000002F49494931000007
:1001F000003C4A4949300000000171090503000034
:10020000003649494936000000064949291E0000C8
:1002100000006C6C000000000000EC6C00000000AE
:10022000000814224100000000242424242400009B
:1002300000004122140800000002015909060000D4
:10024000003E415D551E0000007E1111117E000030
:10025000007F494949360000003E414141220000EB
:10026000007F4141413E0000007F49494941000073
:10027000007F090909010000003E4149497A000058
:10028000007F0808087F00000000417F4100000057
:1002900000304040403F0000007F08142241000031
:1002A000007F404040400000007F0204027F0000C9
:1002B000007F0204087F0000003E4141413E0000F3
:1002C000007F090909060000003E4151215E00003F
:1002D000007F0909196600000026494949320000DB
:1002E0000001017F01010000003F4040403F00004D
:1002F000001F2040201F0000003F403C403F000006
:100300000063140814630000000708700807000069
:10031000007149454300000000007F41410000009A
:100320000002040810200000000041417F0000008E
:1003300000040201020400008080808080808080B0
:10034000000003070000000000205454547800000F
:10035000007F4444443800000038444444280000EE
:1003600000384444447F00000038545454080000CE
:1003700000087E09090000000018A4A4A47C000065
:10038000007F0404780000000000007D40000000B1
:10039000004080847D000000007F102844000000A1
:1003A0000000007F40000000007C0418047800007A
:1003B000007C040478000000003844444438000005
:1003C00000FC4444443800000038444444FC00002D
:1003D00000447844040800000008545454200000ED
:1003E00000043E4424000000003C40207C0000004B
:1003F000001C2040201C0000003C6030603C0000DD
:10040000006C10106C000000009CA0603C0000001C
:10041000006454544C00000000083E4141000000BC
:100420000000007700000000000041413E0800008D
:100430000002010201000000003C2623263C0000CF
:10044000001EA1E121120000003D40207D000000BF
:1004500000385454550900000020555555780000C7
:100460000020555455780000002055555478000060
:100470000020575557780000001CA2E2221400000B
:1004800000385555550800000038555455080000EF
:1004900000385555540800000000017C4100000060
:1004A00000000279420000000000017C40000000D2
:1004B000007029242970000000782F252F78000073
:1004C000007C5454554500000034547C54580000BE
:1004D000007E097F49490000003845453900000089
:1004E0000038454439000000003945443800000018
:1004F000003C41217D000000003D41207C000000C7
:10050000009CA1603D000000003D42423D00000013
:10051000003C41403D00000000182466240000001B
:1005200000483E494962000000292A7C2A2900002F
:10053000007F0916781000000040887E0902000044
:1005400000205455557800000000007D4100000057
:100550000038444539000000003C40217D00000087
:10056000007A090A71000000007A11227900000067
:1005700000085555555E0000004E51514E000000D8
:100580000030484D40200000003C040404040000FA
:1005900004040404041C00000017084C6A50000006
:1005A000001708342A7800000000307D3000000079
:1005B00000081400081400000014080014080000CB
:1005C0004411441144110000AA55AA55AA5500002F
:1005D000BBEEBBEEBBEE0000000000FF0000000021
:1005E000080808FF000000000A0A0AFF00000000D7
:1005F00008FF00FF0000000008F808F800000000F5
:100600000A0A0AFE000000000AFB00FF00000000CA
:1006100000FF00FF000000000AFA02FE00000000D8
:100620000A0B080F00000000080F080F0000000070
:100630000A0A0A0F00000000080808F8000000007D
:100640000000000F080800000808080F0808000054
:10065000080808F808080000000000FF080800006B
:100660000808080808080000080808FF0808000033
:10067000000000FF0A0A000000FF00FF0808000059
:10068000000F080B0A0A000000FE02FA0A0A000026
:100690000A0B080B0A0A00000AFA02FA0A0A00000A
:1006A00000FF00FB0A0A00000A0A0A0A0A0A000000
:1006B0000AFB00FB0A0A00000A0A0A0B0A0A0000E9
:1006C000080F080F080800000A0A0AFA0A0A0000C0
:1006D00008F808F808080000000F080F08080000D4
:1006E0000000000F0A0A0000000000FE0A0A0000D5
:1006F00000F808F80808000008FF00FF08080000DC
:100700000A0A0AFB0A0A00000808080F0000000095
:10071000000000F808080000FFFFFFFFFFFF0000D7
:10072000F0F0F0F0F0F00000FFFFFF00000000002C
:10073000000000FFFFFF00000F0F0F0F0F0F000062
:10074000001824241824000000FE4A4A3400000047
:10075000007F01010300000000027E027E02000013
:100760000063554963000000001824241C040000A5
:1007700000FC20201C000000000804780400000099
:100780000008557755080000003E49493E0000002A
:10079000004C7202724C00000022555930000000DB
:1007A00000182418241800000018247E24180000C3
:1007B000001C2A2A2A000000003C02023C00000023
:1007C000002A2A2A2A0000000000242E240000000B
:1007D00000514A4A4400000000444A4A51000000C7
:1007E000000000FC020400000020403F0000000068
:1007F0000008082A08080000002412241200000043
:10080000000609090600000000001818000000009A
:1008100000000800000000000030403E020200001E
:1008200000010E010E00000000090D0A000000008A
:10083000003C3C3C3C000000ECE3F1E0A0E0B1E017
:10084000ED93FC93A4EEB4E0E2E3F0E094E00E94C8
:10085000A53CE4EEF4E00E944039E6E2FDE70E94A8
:10086000A83A0E94B13A18F011F00C9439040C9493
:100870003F04A4EEB4E0EAE2FDE70E949B3BE4EE15
:10088000F4E00E944039EEE2FDE70E94A83A0E949F
:10089000B13A10F00C945204A4EEB4E0EAE2FDE7A1
:1008A0000E949B3B80E092E2A4E1B1E08D939C9397
:1008B0005A924A92A4E1B1E08D919C91D2018D931C
:1008C0009C9382E00E9498380E942826229682E01B
:1008D0000E948435A6EAB1E0E6EBFDE70E94C93844
:1008E000ACEAB1E0ECEBFDE70E94C938A2EBB1E065
:1008F000E2ECFDE70E94C938A8EBB1E0E8ECFDE7C7
:100900000E94C938AEEBB1E0EEECFDE70E94C938B9
:10091000A4ECB1E0E4EDFDE70E94C938A8EAB4E038
:10092000E2E3FDE70E949B3BACEAB4E0E6E3FDE7CF
:100930000E949B3BA0EBB4E0EAE3FDE70E949B3BF7
:10094000A4EBB4E0EEE3FDE70E949B3BA8EBB4E030
:10095000E2E4FDE70E949B3B82E08093C80483E0D1
:100960008093CB01AAE1B1E0E6E4FDE70E949B3B66
:10097000EAE1F1E00E940239A2E3B1E0EDE0FF27F5
:100980000E94853C85E0809336014091360101E06C
:10099000041718F011F00C94FB04A6E3B1E0AD903D
:1009A000BB24AEE1B1E0AA0CBB1CAA0CBB1CAA0D77
:1009B000BB1D0D911D912D913C914AE050E060E0EE
:1009C00070E00E940A36A6E3B1E0AD90BB24AAE134
:1009D000B1E0AA0CBB1CAA0CBB1CAA0DBB1D4D93FD
:1009E0005D936D937D9380913601815080933601A4
:1009F00010F00C94C504A7E3B1E0E6EBFDE70E941C
:100A0000C938ADE3B1E0ECEBFDE70E94C938A3E4DF
:100A1000B1E0E2ECFDE70E94C938A9E4B1E0E8ECFE
:100A2000FDE70E94C938AFE4B1E0EEECFDE70E94BB
:100A3000C938A5E5B1E0E4EDFDE70E94C93881E0E1
:100A400080935B0102E310E020E030E0A2E3B1E03C
:100A50004D915D916D917C910E94A638ACE5B1E01D
:100A60000D931D932D933D93A2E2B1E00D911D9145
:100A70002D913C91A0E6B1E00D931D932D933C93F5
:100A80007091880170687093880182E08093890179
:100A9000A2E3B1E00D911D912D913C91ACE0B1E04C
:100AA0000D931D932D933C930E94B43782E0809365
:100AB000020181E080930301882780930401EAED1D
:100AC000FDE70E94F73583E08093020181E0809387
:100AD0000301882780930401ECEEFDE70E94F735BF
:100AE00084E08093020181E0809303018827809352
:100AF0000401EEEFFDE70E94F73585E080930201E7
:100B000081E080930301882780930401E0E1FEE700
:100B10000E94F73586E08093020181E08093030113
:100B2000882780930401E2E2FEE70E94F73587E020
:100B30008093020181E08093030188278093040160
:100B4000E4E3FEE70E94F735E2E0F0E00E94FE35C4
:100B50000E94B43703B14EE00423A5E0B1E00C934A
:100B6000009105010A3011F00C940C06A2E3B1E0EB
:100B70000D911D912D913C91A4E6B1E00D931D9333
:100B80002D933C93A2E3B1E00D911D912D913C91E9
:100B9000A8E6B1E00D931D932D933C930EE110E078
:100BA00020E030E0A2E3B1E04D915D916D917C9148
:100BB0000E94A638ACE6B1E00D931D932D933D93B2
:100BC000A6E2B1E00D911D912D913C91A0E7B1E01D
:100BD0000D931D932D933C93A4E7B1E0EAE4FDE768
:100BE0000E949B3BA8E7B1E0EAE4FDE70E949B3B43
:100BF000ACEBB4E0EAE3FDE70E949B3BA0ECB4E081
:100C0000EEE3FDE70E949B3B80E08093E80481E0F7
:100C10008093E9040C945006E0E0F0E0A4E6B1E033
:100C200094E00E94A53CE4E0F0E0A8E6B1E094E0A6
:100C30000E94A53CE8E0F0E0ACE6B1E094E00E9460
:100C4000A53CECE0F0E0A0E7B1E094E00E94A53C18
:100C5000E0E1F0E0A4E7B1E094E00E94A53CE4E12B
:100C6000F0E0A8E7B1E094E00E94A53CACEBB4E072
:100C7000E4E2F0E094E00E94A53CA0ECB4E0E8E2FD
:100C8000F0E094E00E94A53CE7E3F0E0A9EEB4E0D8
:100C90000E94A23CE6E3F0E0A8EEB4E00E94A23C91
:100CA000009105010A3011F00C946B0685E08093E9
:100CB000020181E080930301882780930401E6E428
:100CC000FEE70E94F73503B14EE00423A5E0B1E052
:100CD0000C930C9450060E94B4378AEF90E00E9467
:100CE000673670917A00706870937A00ECE2F0E0F9
:100CF000A2EEB4E00E94A43C0091E904023010F09E
:100D00000C948A0687E68093C40080E08093C50037
:100D10000C94BD06023011F00C94960683E3809388
:100D2000C40080E08093C5000C94BD06033011F030
:100D30000C94A20689E18093C40080E08093C500F2
:100D40000C94BD06043011F00C94AE0680E1809343
:100D5000C40080E08093C5000C94BD060091E904B6
:100D6000043018F011F00C94B7060C94BD0688E01E
:100D70008093C40080E08093C5008AEF90E00E94D9
:100D800067368BE08093CA0181E08093EF01AAEC83
:100D9000B1E0BA93AA930E948327229603B14EE052
:100DA0000423A5E0B1E00C9300910501023011F09D
:100DB0000C94F7060E940635AAECB1E08C918F5F87
:100DC0008C930091CA01073110F40C94EA0687E174
:100DD0008093CA010E94B437AAECB1E0BA93AA93F7
:100DE0000E94832722968AEF90E00E946736009146
:100DF0000501063011F00C941B070E940635809106
:100E0000CA0181508093CA010091CA010B3018F0C9
:100E100011F00C940E078BE08093CA010E94B43746
:100E2000AAECB1E0BA93AA930E94832722968AEF94
:100E300090E00E94673600910501083011F00C9493
:100E400035070E940635AAECB1E0BA93AA930E9436
:100E50007D2E2296AAECB1E0BA93AA930E94832732
:100E600022968AEF90E00E946736009105010C30CF
:100E700011F00C944F070E940635AAECB1E0BA932A
:100E8000AA930E94D3302296AAECB1E0BA93AA9317
:100E90000E94832722968AEF90E00E946736009195
:100EA000CA01073111F00C94B80703B14EE00423D6
:100EB000A5E0B1E00C93009105010A3011F00C940B
:100EC00063070C9465070C945507E0E0F0E0A4E696
:100ED000B1E094E07BE70E94943CE4E0F0E0A8E617
:100EE000B1E094E07BE70E94943CE8E0F0E0ACE6FF
:100EF000B1E094E07BE70E94943CECE0F0E0A0E7F6
:100F0000B1E094E07BE70E94943CE0E1F0E0A4E7EC
:100F1000B1E094E07BE70E94943CE4E1F0E0A8E7D4
:100F2000B1E094E07BE70E94943CE4E2F0E0ACEBBB
:100F3000B4E094E07BE70E94943CE8E2F0E0A0ECAF
:100F4000B4E094E07BE70E94943CE7E3F0E0A9EE94
:100F5000B4E07BE70E94913CE6E3F0E0A8EEB4E069
:100F60007BE70E94913C8BE08093CA010C94BD0604
:100F70000091CA010B3011F00C94742503B14EE0BE
:100F80000423A5E0B1E00C93009105010A3011F0B3
:100F90000C9474250E9406358AEF90E00E94673613
:100FA0000E94B43781E08093020181E080930301C5
:100FB00081E080930401E4E5FEE70E94F73582E0DA
:100FC0008093020181E080930301882780930401CC
:100FD000E4E6FEE70E94F73583E08093020181E0BA
:100FE00080930301882780930401E0E7FEE70E94D5
:100FF000F73584E08093020181E080930301882724
:1010000080930401ECE7FEE70E94F73585E08093CA
:10101000020181E080930301882780930401E8E8BE
:10102000FEE70E94F73586E08093020181E080931D
:101030000301882780930401E0E9FEE70E94F73569
:1010400087E08093020181E08093030188278093E9
:101050000401ECE9FEE70E94F73588E08093020185
:1010600081E080930301882780930401ECEAFEE786
:101070000E94F73503B14EE00423A5E0B1E00C93E4
:1010800000910501063011F00C945B080E940635B2
:101090008091EF0181508093EF017091880170641D
:1010A000709388010091EF01013010F00C945B08FF
:1010B00088E08093EF0100910501023011F00C945B
:1010C00079080E940635AFEEB1E08C918F5F8C936A
:1010D000709188017064709388010091EF0108306D
:1010E00018F011F00C9476080C94790881E0809344
:1010F000EF01A8E8B1E08C9186FB16F00C94FB0B95
:101100000E94B4370091EF01013011F00C94F20805
:1011100081E08093020181E08093030181E080936C
:101120000401E4E5FEE70E94F73582E080930201C6
:1011300081E080930301882780930401E4E6FEE7C1
:101140000E94F73583E08093020181E080930301E0
:10115000882780930401E0E7FEE70E94F73584E0EA
:101160008093020181E0809303018827809304012A
:10117000ECE7FEE70E94F73585E08093020181E00D
:1011800080930301882780930401E8E8FEE70E942A
:10119000F73586E08093020181E080930301882780
:1011A00080930401E0E9FEE70E94F73587E0809331
:1011B000020181E080930301882780930401ECE918
:1011C000FEE70E94F73588E08093020181E080937A
:1011D0000301882780930401ECEAFEE70E94F735BB
:1011E0000C94F20B023011F00C94600981E08093B2
:1011F000020181E080930301882780930401E4E5E4
:10120000FEE70E94F73582E08093020181E080933F
:10121000030181E080930401E4E6FEE70E94F735D4
:1012200083E08093020181E080930301882780930B
:101230000401E0E7FEE70E94F73584E080930201B5
:1012400081E080930301882780930401ECE7FEE7A7
:101250000E94F73585E08093020181E080930301CD
:10126000882780930401E8E8FEE70E94F73586E0CE
:101270008093020181E08093030188278093040119
:10128000E0E9FEE70E94F73587E08093020181E004
:1012900080930301882780930401ECE9FEE70E9414
:1012A000F73588E08093020181E08093030188276D
:1012B00080930401ECEAFEE70E94F7350C94F20BF0
:1012C000033011F00C94CE0981E08093020181E09B
:1012D00080930301882780930401E4E5FEE70E94E0
:1012E000F73582E08093020181E080930301882733
:1012F00080930401E4E6FEE70E94F73583E08093E3
:10130000020181E08093030181E080930401E0E722
:10131000FEE70E94F73584E08093020181E080932C
:101320000301882780930401ECE7FEE70E94F7356C
:1013300085E08093020181E08093030188278093F8
:101340000401E8E8FEE70E94F73586E08093020199
:1013500081E080930301882780930401E0E9FEE7A0
:101360000E94F73587E08093020181E080930301BA
:10137000882780930401ECE9FEE70E94F73588E0B6
:101380008093020181E08093030188278093040108
:10139000ECEAFEE70E94F7350C94F20B043011F0F2
:1013A0000C943C0A81E08093020181E08093030168
:1013B000882780930401E4E5FEE70E94F73582E088
:1013C0008093020181E080930301882780930401C8
:1013D000E4E6FEE70E94F73583E08093020181E0B6
:1013E00080930301882780930401E0E7FEE70E94D1
:1013F000F73584E08093020181E08093030181E06E
:1014000080930401ECE7FEE70E94F73585E08093C6
:10141000020181E080930301882780930401E8E8BA
:10142000FEE70E94F73586E08093020181E0809319
:101430000301882780930401E0E9FEE70E94F73565
:1014400087E08093020181E08093030188278093E5
:101450000401ECE9FEE70E94F73588E08093020181
:1014600081E080930301882780930401ECEAFEE782
:101470000E94F7350C94F20B053011F00C94AA0A77
:1014800081E08093020181E08093030188278093AB
:101490000401E4E5FEE70E94F73582E08093020153
:1014A00081E080930301882780930401E4E6FEE74E
:1014B0000E94F73583E08093020181E0809303016D
:1014C000882780930401E0E7FEE70E94F73584E077
:1014D0008093020181E080930301882780930401B7
:1014E000ECE7FEE70E94F73585E08093020181E09A
:1014F0008093030181E080930401E8E8FEE70E9405
:10150000F73586E08093020181E08093030188270C
:1015100080930401E0E9FEE70E94F73587E08093BD
:10152000020181E080930301882780930401ECE9A4
:10153000FEE70E94F73588E08093020181E0809306
:101540000301882780930401ECEAFEE70E94F73547
:101550000C94F20B063011F00C94180B81E0809380
:10156000020181E080930301882780930401E4E570
:10157000FEE70E94F73582E08093020181E08093CC
:101580000301882780930401E4E6FEE70E94F73513
:1015900083E08093020181E0809303018827809398
:1015A0000401E0E7FEE70E94F73584E08093020142
:1015B00081E080930301882780930401ECE7FEE734
:1015C0000E94F73585E08093020181E0809303015A
:1015D000882780930401E8E8FEE70E94F73586E05B
:1015E0008093020181E08093030181E080930401F4
:1015F000E0E9FEE70E94F73587E08093020181E091
:1016000080930301882780930401ECE9FEE70E94A0
:10161000F73588E08093020181E0809303018827F9
:1016200080930401ECEAFEE70E94F7350C94F20B7C
:10163000073011F00C94860B81E08093020181E069
:1016400080930301882780930401E4E5FEE70E946C
:10165000F73582E08093020181E0809303018827BF
:1016600080930401E4E6FEE70E94F73583E080936F
:10167000020181E080930301882780930401E0E761
:10168000FEE70E94F73584E08093020181E08093B9
:101690000301882780930401ECE7FEE70E94F735F9
:1016A00085E08093020181E0809303018827809385
:1016B0000401E8E8FEE70E94F73586E08093020126
:1016C00081E080930301882780930401E0E9FEE72D
:1016D0000E94F73587E08093020181E08093030147
:1016E00081E080930401ECE9FEE70E94F73588E091
:1016F0008093020181E08093030188278093040195
:10170000ECEAFEE70E94F7350C94F20B083011F07A
:101710000C94F20B81E08093020181E0809303013D
:10172000882780930401E4E5FEE70E94F73582E014
:101730008093020181E08093030188278093040154
:10174000E4E6FEE70E94F73583E08093020181E042
:1017500080930301882780930401E0E7FEE70E945D
:10176000F73584E08093020181E0809303018827AC
:1017700080930401ECE7FEE70E94F73585E0809353
:10178000020181E080930301882780930401E8E847
:10179000FEE70E94F73586E08093020181E08093A6
:1017A0000301882780930401E0E9FEE70E94F735F2
:1017B00087E08093020181E0809303018827809372
:1017C0000401ECE9FEE70E94F73588E0809302010E
:1017D00081E08093030181E080930401ECEAFEE75D
:1017E0000E94F7358AEF90E00E9467367091880179
:1017F0007F7B70938801009105010A3011F00C94F1
:10180000070C8AEF90E00E9467360C94090C0C9448
:101810003A088AEF90E00E9467360091EF010530A8
:1018200011F00C94150C0C940E190091EF01083076
:1018300011F00C94D40E78942C9A70E076BD80E070
:1018400090E09093850080938400A0EFB1E00E9427
:10185000A33BA2EFB1E00E94A33B70916E007160C8
:1018600070936E0070916F00716070936F0086E0EE
:1018700085BD81E0809381000E94B43780E08A9327
:1018800081E38A938FE78A9381E38A9381E08A9345
:101890000E94393880E08093360100913601083784
:1018A00018F011F00C946C0CA6E3B1E08C918A93C3
:1018B00080E38A93A6E3B1E08C918A9385E38A93CF
:1018C00081E08A930E943938A6E3B1E08C918C5E66
:1018D0008C9310F40C944D0C88E08093020181E00D
:1018E00080930301882780930401EEEBFEE70E94BA
:1018F000F735A2EFB1E00D911C91083750E01507C4
:1019000018F011F00C94860C0C94D20EF89480917F
:101910008100887F80938100882785BDEEE4FDE704
:101920000E94A83AE0EFF1E0D190E080FF24002788
:101930000E9464390E940C3AEDE0F0E0A9ECB4E0BA
:101940000E94853CD6B4EE24FF2400270E9464390F
:101950000E949B39E9ECF4E00E9440390E944D3A24
:10196000EDE0F0E0A9ECB4E00E94853CE4EEF4E0A8
:101970000E944539E9ECF4E00E9440390E940C3A9B
:10198000EDE0F0E0A9ECB4E00E94853CE2E5FDE783
:101990000E94A83AE9ECF4E00E9440390E94B6396E
:1019A000EDE0F0E0A9ECB4E00E94853CE9ECF4E065
:1019B0000E944539E6E9F1E00E9440390E943E3A32
:1019C000EDE0F0E0A2E9B1E00E94853CE2E9F1E05F
:1019D0000E94073DEDE0F0E0A2E9B1E00E94853C05
:1019E000E9ECF4E00E944539E2E9F1E00E94403977
:1019F0000E94B639EDE0F0E0A2E9B1E00E94853C3A
:101A0000E2E9F1E00E944039E6E5FDE70E94A83AEC
:101A10000E94B13A18F011F00C94100D0C94160DB0
:101A2000E9ECF4E0A6E9B1E00E94853CE9ECF4E0E1
:101A30000E944539EAE9F1E00E9440390E943E3AAD
:101A4000EDE0F0E0A2E9B1E00E94853CE2E9F1E0DE
:101A50000E94073DEDE0F0E0A2E9B1E00E94853C84
:101A6000E9ECF4E00E944539E2E9F1E00E944039F6
:101A70000E94B639EDE0F0E0A2E9B1E00E94853CB9
:101A8000E2E9F1E00E944039E6E5FDE70E94A83A6C
:101A90000E94B13A18F011F00C94500D0C94560DB0
:101AA000E9ECF4E0AAE9B1E00E94853CE9ECF4E05D
:101AB0000E944039EAE5FDE70E94A83A0E94B13A47
:101AC00010F00C946F0DA6E9B1E0EEE5FDE70E9481
:101AD0009B3BAAE9B1E0EEE5FDE70E949B3BE6E90E
:101AE000F1E00E944539E9ECF4E00E9440390E949F
:101AF0004D3AEDE0F0E0A9ECB4E00E94853CEAE963
:101B0000F1E00E944539E9ECF4E00E9440390E947E
:101B10004D3AEDE0F0E0A9ECB4E00E94853CE2E64D
:101B2000FDE70E94A83AE9ECF4E00E9440390E94E7
:101B3000B639EDE0F0E0A9ECB4E00E94853CE6E6C1
:101B4000FDE70E94A83AE9ECF4E00E9440390E94C7
:101B5000B639EDE0F0E0A0EAB4E00E94853CEAE6A8
:101B6000FDE70E94A83AE0EAF4E00E9440390E94B2
:101B70000C3AEDE0F0E0A0EAB4E00E94853CE0EA37
:101B8000F4E00E94803DEDE0F0E00E940239A9E817
:101B9000B1E0DC9280E080933601009136010F378E
:101BA00018F011F00C94EC0DA6E3B1E08C918A933F
:101BB00089E28A93A6E3B1E08C918A938EE28A93BC
:101BC00080E08A930E943938A6E3B1E08C918F5F60
:101BD0008C9310F40C94CD0D80E0809336014091ED
:101BE000890100913601041718F011F00C94100EC1
:101BF000A6E3B1E08C918A9389E28A93A6E3B1E0EF
:101C00008C918A938EE28A9381E08A930E9439387C
:101C1000A6E3B1E08C918F5F8C9310F40C94EF0DE0
:101C2000A0E8BFE0AF93BF93E9ECF4E00E94403935
:101C30000E94763611E005E0BF91AF910E94C23B51
:101C4000E0E8FFE0A4EDB1E00E94803C83E08093F7
:101C5000020181E080930301882780930401E0ED75
:101C6000FEE70E94F73583E08093020181E08093D4
:101C70000301882780930401E2EEFEE70E94F73516
:101C8000A4EDB1E00E94F1350091E804013011F0BB
:101C90000C94540EECEEFEE70E94DE35A4EDB1E0AC
:101CA0000E94D8350E94E53503B14EE00423A5E03B
:101CB000B1E00C93009105010C3011F00C94700E02
:101CC000EEE6FDE70E94A83AE4EEF4E00E94403917
:101CD0000E943E3AEDE0F0E0A4EEB4E00E94853CC4
:101CE00000910501083011F00C94860EEEE6FDE738
:101CF0000E94A83AE4EEF4E00E9440390E944D3A76
:101D0000EDE0F0E0A4EEB4E00E94853C0091050116
:101D10000A3011F00C94B00EA2E9B1E0E2E3F0E079
:101D200094E00E94A53CE4EEF4E00E944039E2E930
:101D3000F1E00E9445390E94B13A11F40C94A80ECA
:101D4000E2E3F0E0A4EEB4E094E07BE70E94943C90
:101D50002C98F89480E991E00E9467360C94BD06B7
:101D6000E6E9F1E0AAE9B1E00E94853CE9ECF4E0A3
:101D7000A6E9B1E00E94853CA0EFB1E00E94A33B40
:101D8000A2EFB1E00E94A33B80E090E09093850039
:101D90008093840070E076BD789486E085BD81E014
:101DA000809381000C94790C0E94B4370091EF016C
:101DB000043011F00C94DE0E0C940E190091EF011A
:101DC000023018F011F00C94E70E0C940E190091EB
:101DD000EF01023011F00C94160F81E080930201A4
:101DE00081E080930301882780930401E0EFFEE700
:101DF0000E94F73583E08093020181E08093030124
:101E0000882780930401E2E0FFE70E94F73585E030
:101E10008093020181E0809303018827809304016D
:101E2000E4E1FFE70E94F7350C948516033011F0CA
:101E30000C94EC1581E08093020181E08093030112
:101E4000882780930401E6E2FFE70E94F73582E0ED
:101E50008093020181E0809303018827809304012D
:101E6000E2E3FFE70E94F73570918801706170939B
:101E7000880187E08093020181E08093030181E083
:101E800080930401E4E4FFE70E94F73588E0809343
:101E9000020181E080930301882780930401E6E535
:101EA000FFE70E94F73503B14EE00423A5E0B1E05F
:101EB0000C93009105010A3011F00C94610F0C9401
:101EC000C90F00910501023081E008F480E08F9392
:101ED00000910501063081E010F009F080E09F914B
:101EE0008923882311F40C94C70FA8E8B1E08C91E2
:101EF00084FB882780F9809580FBA8E8B1E08C916D
:101F000084F98C93A8E8B1E08C9184FB16F00C94D2
:101F1000A90F87E08093020181E08093030181E0B3
:101F200080930401E4E4FFE70E94F73588E08093A2
:101F3000020181E080930301882780930401E6E594
:101F4000FFE70E94F7358AEF90E00E9467360C9415
:101F5000C70F87E08093020181E080930301882707
:101F600080930401E4E4FFE70E94F73588E0809362
:101F7000020181E08093030181E080930401E6E5A2
:101F8000FFE70E94F7358AEF90E00E9467360C94D5
:101F9000530F8AEF90E00E946736A8E8B1E08C9179
:101FA00084FB16F40C9472115E9A8AEF90E00E9402
:101FB00067360E94B43781E08093020181E080930C
:101FC0000301882780930401E8E6FFE70E94F735C4
:101FD00082E08093020181E080930301882780934F
:101FE0000401EAE7FFE70E94F73583E080930201EE
:101FF00081E080930301882780930401E4E1FFE7F7
:102000000E94F73503B14EE00423A5E0B1E00C9344
:10201000009105010A3011F00C9410100C9412106C
:102020000C94021000917C00007E076000937C00FD
:102030000E94CF38ADEDB4E08D939C93EEE2F0E0DA
:10204000ADEDB4E07BE70E94933CECE2F0E0A2EE61
:10205000B4E00E94A43C8AEF90E00E946736E2E37D
:10206000F1E00E9440390E9464390E949B39E2E706
:10207000FDE70E949F3A0E940C3AEDE0F0E0AEE9E5
:10208000B1E00E94853C5E980E94FB268AEF90E0BA
:102090000E9467360E94B43781E08093020181E09C
:1020A00080930301882780930401ECE8FFE70E94F6
:1020B000F73582E08093020181E080930301882755
:1020C00080930401EEE9FFE70E94F73583E08093F7
:1020D000020181E080930301882780930401E0EBF3
:1020E000FFE70E94F73584E08093020181E080934E
:1020F0000301882780930401E2ECFFE70E94F73593
:1021000085E08093020181E080930301882780931A
:102110000401E4EDFFE70E94F73582E390E0A2EED0
:10212000B4E08D939C9388E08093020181E08093DA
:102130000301882780930401E6EEFFE70E94F7354C
:10214000A0E8BFE0E2EEF4E00E94273C0E94EF35F9
:1021500003B14EE00423A5E0B1E00C93009105012A
:102160000C3011F00C94F010A2EEB4E00E948F3508
:10217000A2EEB4E00D911C91013050E0150710F073
:102180000C94C81081E090E0A2EEB4E08D939C9393
:1021900088E08093020181E0809303018827809387
:1021A0000401E0EDFEE70E94F73588E0809302012C
:1021B00081E080930301882780930401E6EEFFE726
:1021C0000E94F735A0E8BFE0E2EEF4E00E94273C71
:1021D0000E94EF3586E990E00E9467360C94311139
:1021E000083011F00C943111A2EEB4E00E94883551
:1021F000A2EEB4E00D911C91073E53E0150718F0D4
:1022000011F00C9405110C940B1187EE93E0A2EEE3
:10221000B4E08D939C9388E08093020181E08093E9
:102220000301882780930401E0EDFEE70E94F73563
:1022300088E08093020181E08093030188278093E6
:102240000401E6EEFFE70E94F735A0E8BFE0E2EE0A
:10225000F4E00E94273C0E94EF3586E990E00E945E
:102260006736009105010A3011F00C947011ECE210
:10227000F0E0A2EEB4E07BE70E94933C0091E8041A
:10228000013011F00C945611E2EFFFE70E94DE35A9
:10229000A0E8BFE0E2EEF4E00E94273C0E94D635C1
:1022A000E6EFFFE70E94DE350E94E5355E9800917B
:1022B0007C00007E076000937C000E94CF38ADEC6C
:1022C000B4E08D939C93E0E3F0E0ADECB4E07BE709
:1022D0000E94933C8AEF90E00E9467360C94721142
:1022E0000C94A810E2E3F1E00E9440390E946439A6
:1022F0000E949B39E2E7FDE70E949F3A0E940C3A58
:10230000EDE0F0E0AEE9B1E00E94853C5E980E940D
:10231000FB268AEF90E00E9467360E94B437EEE217
:10232000F0E0ADEDB4E00E94A43CECE2F0E0A2EEFF
:10233000B4E00E94A43CE0E3F0E0ADECB4E00E9425
:10234000A43CEDECF4E0D190E080FF2400270E9453
:1023500064390E949B39E6E7FDE70E949F3A0E949C
:102360000C3AEDE0F0E0A0EAB4E00E94853CEDEC30
:10237000F4E0D190E080FF2400270E9464390E949D
:102380009B392F933F934F935F93EDEDF4E0D19002
:10239000E080FF2400270E9464395F914F913F91B4
:1023A0002F910E943E3AEDE0F0E0A4EAB4E00E94F2
:1023B000853CE6E7FDE70E94A83AE4EAF4E00E94E3
:1023C00040390E940C3AEDE0F0E0A4EAB4E00E944B
:1023D000853CEAE3FDE70E94A83AE4EAF4E00E94C3
:1023E00040390E94B639EDE0F0E0A4EAB4E00E9482
:1023F000853CA8E0B1E0EAE3FDE70E949B3BE8E012
:10240000F1E0A4EAB4E00E94333EEDE0F0E0A4EA9B
:10241000B4E00E94853CE2EEF4E0D190E080FF243D
:1024200000270E9464390E949B39E4EAF4E00E948C
:1024300040390E940C3AEDE0F0E0A4EAB4E00E94DA
:10244000853CE2E4FDE70E94A83AE4EAF4E00E9459
:1024500040390E940C3AEDE0F0E0A4EAB4E00E94BA
:10246000853CA0E8BFE0AF93BF93E4EAF4E00E94AC
:1024700040390E94763611E001E0BF91AF910E9491
:10248000C23BE0E8FFE0ABEDB1E00E94803C87E0BA
:102490008093020181E080930301882780930401E7
:1024A000EAEFFFE70E94F735ABEDB1E00E94F135AE
:1024B000E6E0F0E80E94F735EDECF4E0D190E08042
:1024C000FF2400270E9464390E949B39EAE7FDE758
:1024D0000E949F3A0E943E3AEDE0F0E0A4EAB4E0A8
:1024E0000E94853CE6E7FDE70E94A83AE4EAF4E0B2
:1024F0000E9440390E940C3AEDE0F0E0A4EAB4E01A
:102500000E94853CEAE3FDE70E94A83AE4EAF4E091
:102510000E9440390E94B639EDE0F0E0A4EAB4E050
:102520000E94853CE8E0F1E0A4EAB4E00E94333E7A
:10253000EDE0F0E0A4EAB4E00E94853CE2EEF4E0D5
:10254000D190E080FF2400270E9464390E949B39CB
:10255000E4EAF4E00E9440390E940C3AEDE0F0E039
:10256000A4EAB4E00E94853CE2E4FDE70E94A83AB8
:10257000E4EAF4E00E9440390E94B639EDE0F0E070
:10258000A4EAB4E00E94853CA0E8BFE0AF93BF930B
:10259000E4EAF4E00E9440390E94763611E001E05E
:1025A000BF91AF910E94C23BE0E8FFE0ABEDB1E02C
:1025B0000E94803C81E08093020181E080930301CE
:1025C000882780930401EAEFFFE70E94F735ABED1F
:1025D000B1E00E94F135EAE0F0E80E94F73580E0D2
:1025E0008A9380E08A9380E58A9380E08A9381E0F1
:1025F0008A930E94393880E08A9387E38A9380E542
:102600008A9387E38A9381E08A930E9439388EE423
:102610008A9387E38A938EE48A9380E08A9381E0A9
:102620008A930E943938EDEDF4E0D190E080FF24E8
:1026300000270E9464390E949B39EAE7FDE70E9467
:102640009F3A0E943E3AEDE0F0E0A4EAB4E00E9436
:10265000853CEEE7FDE70E94A83AE4EAF4E00E9438
:1026600040390E94B639EDE0F0E0A4EAB4E00E94FF
:10267000853C87E38093E004A0EFB1E00E94A33B98
:1026800003B14EE00423A5E0B1E00C9300910501F5
:102690000A3011F00C9452138AEF90E00E946736D2
:1026A0000C94BD0685E090E00E94673600917C00A6
:1026B000007E076000937C000E94CF38ADECB4E050
:1026C0008D939C93E6E7FDE70E94A83AEDECF4E0D9
:1026D000D190E080FF2400270E9464390E940C3AC8
:1026E000EDE0F0E0AAE1B1E00E94853CADEDB4E0A0
:1026F0004D915C91ADECB4E00D911C910417150760
:1027000010F00C948B13ADEDB4E08D919C91ADEC79
:10271000B4E08D939C93ADECB4E00D911C91ADEDC4
:10272000B4E04D915C91041B150BADECB4E00D933E
:102730001C93E4EAF4E00E944539EDECF4E0D1901A
:10274000E080FF2400270E9464390E94B639EDE042
:10275000F0E0AFECB4E00E94853CEFECF4E00E94C6
:10276000803DEDE0F0E00E940239AFEDB4E0DC9294
:102770008091DF048093E10406E34091DF04041BB1
:10278000AFEDB4E00C934091DF040091E004041736
:1027900011F40C941F144091E0040091DF0404171D
:1027A00010F00C94FA138091E0048093360140916C
:1027B00036010091DF04041718F011F00C94F8139F
:1027C00080E18A93A6E3B1E08C918A938EE38A93A9
:1027D000A6E3B1E08C918A9381E08A930E94393814
:1027E0008091360181508093360110F00C94D713FC
:1027F0000C941F148091E004809336014091DF0413
:1028000000913601041718F011F00C941F1480E1A8
:102810008A93A6E3B1E08C918A938EE38A93A6E330
:10282000B1E08C918A9380E08A930E943938A6E3C4
:10283000B1E08C918F5F8C9310F40C94FE13809117
:10284000DF048093E004E0EAF4E00E944539EAE125
:10285000F1E00E9440390E943E3AEDE0F0E0AAE14A
:10286000B1E00E94853CEAE3FDE70E94A83AEAE174
:10287000F1E00E9440390E94B639EDE0F0E0AAE1B3
:10288000B1E00E94853CA8E0B1E0EAE3FDE70E94E8
:102890009B3BE8E0F1E0AAE1B1E00E94333EEDE0CD
:1028A000F0E0AAE1B1E00E94853CEAE1F1E00E949B
:1028B0004539E2EEF4E0D190E080FF2400270E9449
:1028C00064390E940C3AEDE0F0E0AAE1B1E00E9428
:1028D000853C8AE090E00E946736A0EFB1E00D9160
:1028E0001C910D3250E0150711F00C94DC15A0EF8F
:1028F000B1E00E94A33B88E08093020181E08093D5
:102900000301882780930401E0EDFEE70E94F7357C
:10291000EAE1F1E00E94863EEDE0F0E0A8E0B1E0FF
:102920000E94853CE8E0F1E00E944539EAE3FDE7DA
:102930000E949F3A0E940C3AEDE0F0E0A8E0B1E07E
:102940000E94853CA0E8BFE0AF93BF93E8E0F1E0D0
:102950000E9440390E94763611E001E0BF91AF91AC
:102960000E94C23BE0E8FFE0A4EDB1E00E94803CA1
:10297000EAE1F1E00E944039E2E4FDE70E94A83A72
:102980000E94B13A10F00C947B15EAE1F1E00E944C
:102990004039E6E3FDE70E94A83A0E94B13A18F0F8
:1029A00011F00C94D5140C942815A0E8BFE0AF9357
:1029B000BF93EAE1F1E00E9440390E94763611E0CF
:1029C00001E0BF91AF910E94C23BE0E8FFE0ABEDB8
:1029D000B1E00E94803C88E08093020181E0809316
:1029E0000301882780930401ABEDB1E00E94F1352B
:1029F000EEE0F0E80E94F735A4EDB1E00E94F13579
:102A0000E2E1F0E80E94F7350091E804013011F0AE
:102A10000C942615E6E1F0E80E94DE35ABEDB1E05E
:102A20000E94D835E6EFFFE70E94DE350E94E535CB
:102A3000EAE1F0E80E94DE35A4EDB1E00E94D8356D
:102A4000EEE1F0E80E94DE350E94E5350C94791540
:102A5000A0E8BFE0AF93BF93EAE1F1E00E94403904
:102A60000E94763611E003E0BF91AF910E94C23B15
:102A7000E0E8FFE0ABEDB1E00E94803C88E08093AD
:102A8000020181E080930301882780930401ABED6C
:102A9000B1E00E94F135EEE0F0E80E94F735A4EDD8
:102AA000B1E00E94F135E2E1F0E80E94F7350091D3
:102AB000E804013011F00C947915E6E1F0E80E9489
:102AC000DE35ABEDB1E00E94D835E6EFFFE70E94BE
:102AD000DE350E94E535EAE1F0E80E94DE35A4ED3E
:102AE000B1E00E94D835EEE1F0E80E94DE350E94A8
:102AF000E5350C94DC15E2E4FDE70E94A83AEAE132
:102B0000F1E00E9440390E94B639EDE0F0E0AAE120
:102B1000B1E00E94853CA0E8BFE0AF93BF93EAE13B
:102B2000F1E00E9440390E94763611E001E0BF9149
:102B3000AF910E94C23BE0E8FFE0ABEDB1E00E9444
:102B4000803C88E08093020181E080930301882724
:102B500080930401ABEDB1E00E94F135EAE0F0E8CA
:102B60000E94F735A4EDB1E00E94F135E2E1F0E812
:102B70000E94F7350091E804013011F00C94DC1547
:102B8000E6E1F0E80E94DE35ABEDB1E00E94D83519
:102B9000E2E2F0E80E94DE350E94E535EAE1F0E885
:102BA0000E94DE35A4EDB1E00E94D835EEE1F0E8F8
:102BB0000E94DE350E94E535A0EFB1E00D911C9139
:102BC00041E050E0040F151FA0EFB1E00D931C93FE
:102BD0000C9440130C948516063011F00C941916C1
:102BE00081E08093020181E0809303018827809334
:102BF0000401E0EFFEE70E94F73583E080930201D5
:102C000081E080930301882780930401E2E0FFE7DD
:102C10000E94F73585E08093020181E080930301F3
:102C2000882780930401E4E1FFE70E94F7350C94C4
:102C30008516073011F00C94851681E0809302010F
:102C400081E080930301882780930401E4E2F0E8A7
:102C50000E94F73582E08093020181E080930301B6
:102C6000882780930401E6E3F0E80E94F73583E0CB
:102C70008093020181E080930301882780930401FF
:102C8000E8E4F0E80E94F73584E08093020181E0F7
:102C900080930301882780930401EAE5F0E80E940D
:102CA000F73585E08093020181E080930301882756
:102CB00080930401ECE6F0E80E94F73586E080930B
:102CC000020181E080930301882780930401EEE7ED
:102CD000F0E80E94F73587E08093020181E080935D
:102CE0000301882780930401E0E9F0E80E94F735AA
:102CF00088E08093020181E080930301882780931C
:102D00000401E2EAF0E80E94F73503B14EE0042343
:102D1000A5E0B1E00C93009105010A3011F00C948C
:102D200093160C9497160E9406350C9485160E94F3
:102D30007625A0EFB1E00E94A33BA0EFB1E00D919A
:102D40001C910F3750E0150718F011F00C94CE16B7
:102D500080E380933601009136010A3318F011F0B8
:102D60000C94C316A0EFB1E04C91A6E3B1E05C91E6
:102D700091E00E941238A6E3B1E08C918F5F8C93B2
:102D800010F40C94AB168AE090E00E946736A0EF36
:102D9000B1E00E94883510F40C949D16A5EFB2E0C6
:102DA000E0E8F0E00E94D43CAAE7B4E00D931C9365
:102DB0000E94B4370091EF01023011F00C94161705
:102DC00081E08093020181E0809303018827809352
:102DD0000401E4EBF0E80E94F73583E08093020100
:102DE00081E080930301882780930401E6ECF0E8FA
:102DF0000E94F73584E08093020181E08093030113
:102E0000882780930401E8EDF0E80E94F73586E01A
:102E10008093020181E0809303018827809304015D
:102E2000E4E1FFE70E94F7350C947B17063011F0C0
:102E30000C94431781E08093020181E080930301A9
:102E4000882780930401E0EFFEE70E94F73583E0D6
:102E50008093020181E0809303018827809304011D
:102E6000EAEEF0E80E94F73585E08093020181E008
:102E700080930301882780930401E4E1FFE70E9427
:102E8000F7350C947B17073011F00C947B1781E019
:102E90008093020181E080930301882780930401DD
:102EA000ECEFF0E80E94F73583E08093020181E0C7
:102EB00080930301882780930401EEE0F1E80E94EB
:102EC000F73584E08093020181E080930301882735
:102ED00080930401E0E9F0E80E94F73586E08093F2
:102EE000020181E080930301882780930401E4E1DB
:102EF000FFE70E94F73503B14EE00423A5E0B1E0FF
:102F00000C93009105010A3011F00C9489170C9470
:102F10008D170E9406350C947B170E947625A0EF32
:102F2000B1E00E94A33BA0EFB1E00D911C910F37DF
:102F300050E0150718F011F00C94C41780E380934B
:102F40003601009136010A3318F011F00C94B917CC
:102F5000A0EFB1E04C91A6E3B1E05C9191E00E945A
:102F60001238A6E3B1E08C918F5F8C9310F40C942F
:102F7000A1178AE090E00E946736A0EFB1E00E94BE
:102F8000883510F40C9493170E94B4370091EF0128
:102F9000023011F00C94F51781E08093020181E07A
:102FA00080930301882780930401E0E2F1E80E9406
:102FB000F73583E08093020181E080930301882745
:102FC00080930401E0E3F1E80E94F73584E0809308
:102FD000020181E080930301882780930401E0E4EB
:102FE000F1E80E94F7350C944D18063011F00C945E
:102FF000221881E08093020181E0809303018827F9
:1030000080930401E0E2F1E80E94F73583E08093C9
:10301000020181E080930301882780930401E0E5A9
:10302000F1E80E94F73584E08093020181E080930B
:103030000301882780930401EEE5F1E80E94F7354B
:103040000C944D18073011F00C944D1881E08093CA
:10305000020181E080930301882780930401E0E26C
:10306000F1E80E94F73583E08093020181E08093CC
:103070000301882780930401E0E5F1E80E94F73519
:1030800084E08093020181E080930301882780938C
:103090000401EEE5F1E80E94F735E2E0F0E00E947D
:1030A000FE35A5EFB2E0E0E8F0E00E94C83CA8E7FA
:1030B000B4E00D931C930E94B43781E08093020129
:1030C00081E080930301882780930401E0E2F1E826
:1030D0000E94F73585E08093020181E0809303012F
:1030E000882780930401E2E2FEE70E94F73586E03C
:1030F0008093020181E0809303018827809304017B
:10310000ECE6F1E80E94F735A0E8BFE0EAE7F4E07A
:103110000E94273C0E94EF3587E08093020181E006
:1031200080930301882780930401E4E7F1E80E947B
:10313000F735A0E8BFE0E8E7F4E00E94273C0E94F2
:10314000EF35A8E7B4E00D911C91AAE7B4E04D91EA
:103150005C91041B150BA6E8B4E00D931C93E6E705
:10316000FDE70E94A83AE6E8F4E0D190E080FF2471
:1031700000270E9464390E940C3AEDE0F0E0AEE7CF
:10318000B4E00E94853CE2E8FDE70E94A83AE6E848
:10319000F4E0D190E080FF2400270E9464390E946F
:1031A000B639EDE0F0E0A8E8B4E00E94853CE2E842
:1031B000FDE70E94A83AEEE7F4E00E9440390E9441
:1031C000B639EDE0F0E0A2E8B4E00E94853C88E08A
:1031D0008093020181E0809303018827809304019A
:1031E000ECE7F1E80E94F735EEE7F4E00E94803D5D
:1031F000DD2CEE2CFF2C002FA0E8BFE0EDE0F0E08E
:103200000E9440390E9476360E94EF35E4E8F1E8EA
:103210000E94F735E2E0F0E00E94FE350091EF01F8
:10322000053011F00C94B91980E890E0A2EEB4E0FA
:103230008D939C93ACE6B1E00D911D912D913C9145
:10324000A8E6B1E04D915D916D917C910E940F3C9B
:10325000AEE8B1E00D931D932D933D93A2EEB4E043
:103260000D911C912227332749EF54E160E070E073
:103270000E94A638A9EDB4E00D931D932D933D93C4
:10328000AEE8B1E04D915D916D917C91A9EDB4E016
:103290000D911D912D913C910E94143C1CF011F058
:1032A0000C94721902E010E0A2EEB4E04D915C9132
:1032B0000E949C38A2EEB4E00D931C93A2EEB4E001
:1032C0000D911C912227332749EF54E160E070E013
:1032D0000E94A638A9EDB4E00D931D932D933D9364
:1032E0000C944019AEE8B1E00D911D912D913C91E7
:1032F000A2EEB4E04D915C91662777270E940A36D2
:10330000A9EDB4E04D935D936D937D93A2EEB4E08F
:103310000D911C9140E850E00E94BC35ADEDB4E049
:103320004D935C93ADEDB4E00D911C91013050E0F4
:10333000150718F011F00C949F190C94AD19ADED10
:10334000B4E00D911C9142E050E00E94BC35ADEC20
:10335000B4E04D935C930C94B519ADEDB4E08D9150
:103360009C91ADECB4E08D939C93A3EDB4E00E94EE
:10337000A33B0E94B43787E090E0A0E9B4E08D93CE
:103380009C93ACE8B4E00E94A33BA0EFB1E00E94A4
:10339000A33B709188017B7F7093880103B14EE05D
:1033A0000423A5E0B1E00C93A0EFB1E00E948835C2
:1033B000A0EFB1E00D911C910F3750E0150718F008
:1033C00011F00C94E5190C94A51DA0EFB1E00E943A
:1033D000A33BA8E8B1E08C9182FB16F00C94F7199E
:1033E000709188017B7F709388010E94B437ACE8AC
:1033F000B4E08C918A9380E08A93ACE8B4E08C913D
:103400008A938FE38A9381E08A930E94393880E01F
:103410008A93A0E9B4E08C918A938FE78A93A0E91C
:10342000B4E08C918A9381E08A930E9439380E949B
:1034300060330091EF01053011F00C94471A81E0E0
:103440008093020181E08093030188278093040127
:10345000E0EDFEE70E94F73581E08093020181E014
:1034600080930301882780930401A4EDB1E00E94BA
:10347000F135E8E8F1E80E94F735A7E9B4E00E94E9
:10348000F135ECE8F1E80E94F7350C946D1A88E00C
:103490008093020181E080930301882780930401D7
:1034A000E0EDFEE70E94F73588E08093020181E0BD
:1034B00080930301882780930401A4EDB1E00E946A
:1034C000F135E8E8F1E80E94F735A7E9B4E00E9499
:1034D000F135ECE8F1E80E94F7350091EF01073093
:1034E00081E009F080E08F930091EF01043081E0EA
:1034F00009F080E09F91892B882311F40C94381BEC
:1035000070918801706470938801E3E9F4E00E948F
:103510004039E6E8FDE70E94A83A0E94B13A10F46B
:103520000C949A1AA4EDB1E0E0E9F1E80E94C938E0
:103530000C941A1BA7E9B4E00E94C73AEDE0F0E052
:10354000A0EAB4E00E94853CEAE8FDE70E94A83AC0
:10355000E0EAF4E00E9440390E940C3AEDE0F0E02D
:10356000A0EAB4E00E94853CEEE8FDE70E94A83A9C
:10357000E0EAF4E00E9440390E94B639EDE0F0E064
:10358000A0EAB4E00E94853CE0EAF4E00E944539FC
:10359000EAE3FDE70E949F3A0E94203EEDE0F0E062
:1035A000A4EAB4E00E94853CE6E3FDE70E94A83A65
:1035B000E4EAF4E00E9440390E944D3AEDE0F0E088
:1035C000A0EAB4E00E94853CE6E3FDE70E94A83A49
:1035D000E4EAF4E00E9440390E943E3AEDE0F0E077
:1035E000A4EAB4E00E94853CE4EAF4E00E94453994
:1035F000E0EAF4E00E9440390E94B639EDE0F0E0E4
:10360000A0EAB4E00E94853CA0E8BFE0AF93BF937E
:10361000E0EAF4E00E9440390E94763611E002E0D0
:10362000BF91AF910E94C23BE0E8FFE0A4EDB1E0A2
:103630000E94803C81E08093020181E0809303013D
:10364000882780930401E0EDFEE70E94F73581E0D2
:103650008093020181E08093030188278093040115
:10366000E4E9F1E80E94F735A4EDB1E00E94F135FC
:103670000091EF01023011F00C949C1DA5EFB1E018
:10368000E0E8F0E00E94E03CADECB4E00D931C9368
:10369000A5EDB4E04D935C9387E08093020181E057
:1036A00080930301882780930401E0EAF1E80E94F7
:1036B000F735A0E8BFE0EDECF4E00E94273C0E9463
:1036C000EF3586E08093020181E080930301882733
:1036D00080930401E6EAF1E80E94F735A0E8BFE034
:1036E000E5EDF4E00E94273C0E94EF35ADECB4E03C
:1036F0000D911C914FE050E0040F151FA3EDB4E0B5
:103700000D931C938091D50480933601409136012E
:1037100001E0041718F011F00C94B01BA3EDB4E015
:103720004D915C91A6E3B1E0AD90BB24A3EFB1E075
:10373000AA0CBB1CAA0DBB1D0D911C9104171507EB
:1037400018F011F00C94A61B0C94A81B0C94B01B41
:103750008091360181508093360110F00C94861BC5
:10376000809136018093D7048091D50480933601EF
:10377000009136010F3718F011F00C94E11BA3ED06
:10378000B4E04D915C91A6E3B1E0AD90BB24A3EF12
:10379000B1E0AA0CBB1CAA0DBB1D0D911C91041716
:1037A000150718F011F00C94D71B0C94D91B0C942E
:1037B000E11BA6E3B1E08C918F5F8C9310F40C9425
:1037C000B81B809136018093D804A8EDB4E00C9129
:1037D000112722273327A7EDB4E04C915527662700
:1037E00077270E940F3CA9EDB4E00D931D932D9314
:1037F0003D93A9EDB4E00D911D912D913C91A0E177
:10380000B1E04D915D916D917C910E94A638A9ED3A
:10381000B4E00D931D932D933D930091D8044091F6
:10382000D704040FA7EDB4E00C93A7EDB4E00C911E
:1038300042E00E94B83C0C93E5EDF4E0D190E080CA
:10384000FF2400270E9464390E949B392F933F93E5
:103850004F935F93E0E1F1E00E9440390E946439A8
:103860005F914F913F912F910E940C3AEDE0F0E073
:10387000A9ECB4E00E94853CE9ECF4E00E944539F3
:10388000E8E6F1E00E9440390E9464390E944D3A16
:10389000EDE0F0E0A9ECB4E00E94853CE2E3F1E069
:1038A0000E9440390E9464390E949B39E9ECF4E09F
:1038B0000E9440390E94B639EDE0F0E0ABEEB1E095
:1038C0000E94853CA0E8BFE0AF93BF93EBEEF1E030
:1038D0000E9440390E94763611E005E0BF91AF9119
:1038E0000E94C23BE0E8FFE0A4EDB1E00E94803C12
:1038F00087E08093020181E0809303018827809311
:103900000401ECEAF1E80E94F735A4EDB1E00E9471
:10391000F135E0EBF1E80E94F735E2E3F1E00E94D7
:1039200040390E9464390E949B392F933F934F93F3
:103930005F93E9EDF4E00E9440390E9464395F91A1
:103940004F913F912F910E94B639EDE0F0E0A9EC44
:10395000B4E00E94853CE9ECF4E00E944539EBEECE
:10396000F1E00E9440390E94B639EDE0F0E0A9ECA8
:10397000B4E00E94853CE9ECF4E00E94803DEDE07B
:10398000F0E0A9ECB4E00E94853C84E08093020161
:1039900081E080930301882780930401E4EBF1E840
:1039A0000E94F735A0E8BFE0E9ECF4E00E9440395E
:1039B0000E9476360E94EF35EBEEF1E00E94453929
:1039C000EBEEF1E00E9440390E940C3AEDE0F0E0AD
:1039D000ABEEB1E00E94853CE2E9FDE70E94A83A27
:1039E000EBEEF1E00E9440390E940C3AEDE0F0E08D
:1039F000ABEEB1E00E94853CE0ECF4E00E9445397A
:103A0000EBEEF1E00E9440390E940C3AEDE0F0E06C
:103A1000A9ECB4E00E94853CE6E9FDE70E94A83AE3
:103A2000E9ECF4E00E9440390E940C3AEDE0F0E04D
:103A3000A9ECB4E00E94853CE9ECF4E00E94453931
:103A4000E6E3FDE70E949F3A0E94B639EDE0F0E020
:103A5000A9ECB4E00E94853CA0E8BFE0AF93BF931F
:103A6000E9ECF4E00E9440390E94763611E001E072
:103A7000BF91AF910E94C23BE0E8FFE0A4EDB1E04E
:103A80000E94803C85E08093020181E080930301E5
:103A9000882780930401E8EBF1E80E94F735A4ED54
:103AA000B1E00E94F135ECEBF1E80E94F735ECEB68
:103AB000F4E00E944539EBEEF1E00E9440390E94AB
:103AC0000C3AEDE0F0E0A9ECB4E00E94853CE9ECB2
:103AD000F4E00E944539E2E5FDE70E949F3A0E942A
:103AE000B639EDE0F0E0A9ECB4E00E94853CE9ECE9
:103AF000F4E00E94803DEDE0F0E0A9ECB4E00E942B
:103B0000853C86E08093020181E080930301882751
:103B100080930401E0ECF1E80E94F735A0E8BFE0F3
:103B2000E9ECF4E00E9440390E9476360E94EF35BD
:103B3000E4ECF1E80E94F735A8E8B1E08C9185FB50
:103B400016F00C94A51D0E9460330091EF01053022
:103B500011F40C94481E41E050E060E070E0A8E7EA
:103B6000B1E00D911D912D913C910E94143C11F0FA
:103B70000C94EE1DEAE8F1E00E9440390E9464399D
:103B80000E949B392F933F934F935F93E0EFF1E0B7
:103B9000D190E080FF2400270E9464395F914F910B
:103BA0003F912F910E940C3AEDE0F0E0AEE9B1E0D8
:103BB0000E94853CEEE9F1E00E944539E8E6F1E03B
:103BC0000E9440390E9464390E944D3AEDE0F0E0D5
:103BD000AEE9B1E00E94853C0C942E1EE0EFF1E0CE
:103BE000D190E080FF2400270E9464390E949B3915
:103BF000E2E9F1E00E9440390E940C3AEDE0F0E089
:103C0000AAE9B1E00E94853CE6E9F1E00E9445396D
:103C1000EAE9F1E00E9440390E944D3AEDE0F0E01F
:103C2000AAE9B1E00E94853CEAE9F1E00E94453949
:103C3000EAE3FDE70E949F3A0E94203EEDE0F0E0BB
:103C4000AAE9B1E00E94853CEAE9F1E00E94803DEA
:103C5000EDE0F0E0AEE9B1E00E94853C0E94FB2679
:103C6000A0EFB1E00D911C91003050E0150711F06C
:103C70000C94401E85E090E00E9467360C94481E2C
:103C8000EF93FF93ECE1F3E00E945E36FF91EF913A
:103C9000A0EFB1E00D911C9141E050E0040F151F21
:103CA000A2EFB1E00D931C930091EF01053011F0EC
:103CB0000C94AA1FA0EFB1E00D911C91013050E0CF
:103CC000150781E008F480E08F93A0EFB1E00D913B
:103CD0001C910E3750E0150781E010F009F080E0EC
:103CE0009F918923882311F40C94091FA2EFB1E05E
:103CF000AD90BC90A3EFB1E0AA0CBB1CAA0DBB1DFC
:103D00000E94A33B81E080933601ADEDB4E04D917C
:103D10005C91A6E3B1E00D9111270417150718F087
:103D200011F00C94071FE9EDF4E00E9440390E9465
:103D300064390E949B392F933F934F935F93E3ED38
:103D4000F4E0D190E080FF2400270E9464395F9165
:103D50004F913F912F910E940C3AEDE0F0E0AEE9D7
:103D6000B1E00E94853CEEE9F1E00E944539E8E6C9
:103D7000F1E00E9440390E9464390E944D3AEDE022
:103D8000F0E0AEE9B1E00E94853C0E94FB26A3ED85
:103D9000B4E00E94883500917C00007E07600093AB
:103DA0007C000E94CF38A2EEB4E08D939C93A2EFEA
:103DB000B1E0AD90BC90A3EFB1E0AA0CBB1CAA0D82
:103DC000BB1D4D915C91A2EEB4E00D911C910417C6
:103DD000150718F011F00C94EF1E0C94FF1EA2EEC4
:103DE000B4E08D919C91A2EFB1E0AD90BC90A3EFB7
:103DF000B1E0AA0CBB1CAA0DBB1D8D939C93A6E33E
:103E0000B1E08C918F5F8C9310F40C94851E0C9410
:103E1000A81FA2EFB1E0AD90BC90A3EFB1E0AA0C57
:103E2000BB1CAA0DBB1D0E94A33B81E08093360101
:103E3000ADECB4E04D915C91A6E3B1E00D9111279A
:103E40000417150718F011F00C949A1FE9EDF4E02F
:103E50000E9440390E9464390E949B392F933F93FE
:103E60004F935F93E3EDF4E0D190E080FF240027CF
:103E70000E9464395F914F913F912F910E940C3ABB
:103E8000EDE0F0E0AEE9B1E00E94853CEEE9F1E062
:103E90000E944539E8E6F1E00E9440390E94643909
:103EA0000E944D3AEDE0F0E0AEE9B1E00E94853CC1
:103EB0000E94FB26A3EDB4E00E94883500917C00AF
:103EC000007E076000937C000E94CF38A2EEB4E031
:103ED0008D939C93A2EFB1E0AD90BC90A3EFB1E0C5
:103EE000AA0CBB1CAA0DBB1D4D915C91A2EEB4E0C7
:103EF0000D911C910417150718F011F00C94821FF6
:103F00000C94921FA2EEB4E08D919C91A2EFB1E0CF
:103F1000AD90BC90A3EFB1E0AA0CBB1CAA0DBB1DD9
:103F20008D939C93A6E3B1E08C918F5F8C9310F4FA
:103F30000C94181FA0EFB1E00D911C910F3750E0C9
:103F4000150711F00C94A81FA3EDB4E00E94A33B49
:103F50000C94BE1F00917C00007E076000937C00E3
:103F60000E94CF38A2EFB1E0AD90BC90A3EFB1E0DA
:103F7000AA0CBB1CAA0DBB1D8D939C93A2EFB1E0B4
:103F8000AD90BC90A3EFB2E0AA0CBB1CAA0DBB1D68
:103F90004D915C91A2EFB1E0AD90BC90A3EFB1E088
:103FA000AA0CBB1CAA0DBB1D0D911C910417150773
:103FB00018F011F00C94DE1F0C94F61FA2EFB1E084
:103FC000AD90BC90A3EFB2E0AA0CBB1CAA0DBB1D28
:103FD0008D919C91A2EFB1E0AD90BC90A3EFB1E0C8
:103FE000AA0CBB1CAA0DBB1D8D939C93AAE7B4E041
:103FF0004D915C91A2EFB1E0AD90BC90A3EFB1E028
:10400000AA0CBB1CAA0DBB1D0D911C910417150712
:1040100010F00C941B20AAE7B4E08D919C91A2EFC4
:10402000B1E0AD90BC90A3EFB1E0AA0CBB1CAA0D0F
:10403000BB1D8D939C93A2EFB1E0AD90BC90A3EF1C
:10404000B2E0AA0CBB1CAA0DBB1D0D911C91A2EFE6
:10405000B1E0AD90BC90A3EFB1E0AA0CBB1CAA0DDF
:10406000BB1D4D915C91041B150BACE9B4E00D93A5
:104070001C93E8E8F4E00E944539ECE9F4E0D190C3
:10408000E080FF2400270E9464390E94B639EDE0E9
:10409000F0E0ABEEB1E00E94853CEBEEF1E00E9477
:1040A000803DEDE0F0E00E940239ACE9B4E0DD9241
:1040B000EC92ACE9B4E00D911C9147E050E0040FA4
:1040C000151FACE9B4E00D931C93ACE9B4E00D917D
:1040D0001C91003050E0150710F00C947320ACE9EF
:1040E000B4E00E94A33BACE9B4E00D911C910F3306
:1040F00050E0150718F011F00C9480200C948620E5
:104100008FE390E0ACE9B4E08D939C930091EF01D4
:10411000053011F00C94BF200FE74091F001041B13
:10412000A4EFB1E00C93A4EFB1E08C918A938FE3FC
:104130008A93A4EFB1E08C918A93A2EFB1E0AD90A5
:10414000BC90A4EFB3E0AA0DBB1D8C918A9380E0D4
:104150008A930E943938A4EFB1E08C918A938FE35F
:104160008A93A4EFB1E08C918A93ACE9B4E08C918E
:104170008A9381E08A930E9439380C94D720A0EF6B
:10418000B1E04C91A2EFB1E0AD90BC90A4EFB3E0F0
:10419000AA0DBB1D5C9190E00E941238A0EFB1E027
:1041A0004C91ACE9B4E05C9191E00E9412388091AE
:1041B0009C04A2EFB1E0AD90BC90A4EFB3E0AA0DD7
:1041C000BB1D8C93009105010A3011F00C94EA207C
:1041D0000C94BD06009105010C3011F00C94642282
:1041E0000E940635ACE8B4E08C918A9380E08A9313
:1041F000ACE8B4E08C918A938FE38A9380E08A9351
:104200000E943938ACE8B4E00E948F35ACE8B4E0E5
:104210000D911C91003050E015070CF402C00C9475
:104220009021ACE8B4E00E94A33B709188017460D7
:1042300070938801ACE6B1E00D911D912D913C91F8
:10424000A8E6B1E04D915D916D917C910E940F3C8B
:10425000ACE0B1E00D931D932D933D93ACE0B1E044
:104260000D911D912D913C914AE050E060E070E08D
:104270000E940A36ACE0B1E04D935D936D937D935F
:10428000A8E6B1E00D911D912D913C91ACE0B1E01B
:104290004D915D916D917C910E940F3CA8E6B1E03B
:1042A0000D931D932D933D93A0E6B1E04D915D914B
:1042B0006D917C91A8E6B1E00D911D912D913C91FD
:1042C0000E94143C0CF402C00C947C21A8E6B1E0DE
:1042D0000D911D912D913C91ACE0B1E04D915D911E
:1042E0006D917C910E940A3CA8E6B1E00D931D936C
:1042F0002D933D930C949021ACE6B1E00D911D916E
:104300002D913C91ACE0B1E04D915D916D917C912E
:104310000E940F3CACE6B1E00D931D932D933D93AD
:10432000ACE8B4E08C918A9380E08A93ACE8B4E086
:104330008C918A938FE38A9381E08A930E94393823
:1043400080E08A93A0E9B4E08C918A938FE78A9306
:10435000A0E9B4E08C918A9381E08A930E94393875
:104360000091EF01053011F40C94D72180E0809387
:104370009204009192040F3718F011F00C94D72199
:10438000A2E9B4E04C91A2E9B4E0AD90BB24A5EF62
:10439000B3E0AA0DBB1D5C9191E00E941238A2E926
:1043A000B4E08C918F5F8C9310F40C94B921009140
:1043B000EF01053011F00C940F22EAE8F1E00E94C1
:1043C00040390E9464390E949B392F933F934F9349
:1043D0005F93E4EFF1E0D080EE24FF2400270E94F9
:1043E00064395F914F913F912F910E940C3AEDE01B
:1043F000F0E0AEE9B1E00E94853CEEE9F1E00E9418
:104400004539E8E6F1E00E9440390E9464390E9493
:104410004D3AEDE0F0E0AEE9B1E00E94853C0E944B
:1044200060330091EF01053011F00C94322281E0ED
:104430008093020181E08093030188278093040127
:10444000A4EDB1E00E94F135E8ECF1E80E94F73507
:10445000A7E9B4E00E94F135ECE8F1E80E94F735F5
:104460000C944B2288E08093020181E08093030149
:10447000882780930401A4EDB1E00E94F135E8ECB7
:10448000F1E80E94F735A7E9B4E00E94F135ECE8C5
:10449000F1E80E94F73584E690E00E94673603B1A8
:1044A0004EE00423A5E0B1E00C93009105010C302F
:1044B00011F00C945F220E9406350C94F22070914A
:1044C000880170627093880100910501083011F035
:1044D0000C94E2230E940635ACE8B4E08C918A93F8
:1044E00080E08A93ACE8B4E08C918A938FE38A935E
:1044F00080E08A930E943938ACE8B4E00E948835A5
:10450000ACE8B4E00D911C910F3750E015071CF09A
:1045100011F00C948D220C9410238FE790E0ACE8FE
:10452000B4E08D939C9370918801746070938801BE
:10453000ACE6B1E00D911D912D913C91A8E6B1E062
:104540004D915D916D917C910E940F3CACE0B1E08A
:104550000D931D932D933D93ACE0B1E00D911D9112
:104560002D913C914AE050E060E070E00E940A36F4
:10457000ACE0B1E04D935D936D937D93ACE6B1E01B
:104580000D911D912D913C91ACE0B1E04D915D916B
:104590006D917C910E940A3CACE6B1E00D931D93B5
:1045A0002D933D93ACE5B1E04D915D916D917C9182
:1045B000ACE6B1E00D911D912D913C910E94143C0F
:1045C0001CF011F00C94E6220C94FC22ACE6B1E055
:1045D0000D911D912D913C91ACE0B1E04D915D911B
:1045E0006D917C910E940F3CACE6B1E00D931D9360
:1045F0002D933D930C941023A8E6B1E00D911D91ED
:104600002D913C91ACE0B1E04D915D916D917C912B
:104610000E940A3CA8E6B1E00D931D932D933D93B3
:10462000ACE8B4E08C918A9380E08A93ACE8B4E083
:104630008C918A938FE38A9381E08A930E94393820
:1046400080E08A93A0E9B4E08C918A938FE78A9303
:10465000A0E9B4E08C918A9381E08A930E94393872
:104660000091EF01053011F40C94572380E0809302
:104670009204009192040F3718F011F00C94572314
:10468000A2E9B4E04C91A2E9B4E0AD90BB24A5EF5F
:10469000B3E0AA0DBB1D5C9191E00E941238A2E923
:1046A000B4E08C918F5F8C9310F40C9439230091BB
:1046B000EF01053011F00C948F23EAE8F1E00E943D
:1046C00040390E9464390E949B392F933F934F9346
:1046D0005F93E4EFF1E0D080EE24FF2400270E94F6
:1046E00064395F914F913F912F910E940C3AEDE018
:1046F000F0E0AEE9B1E00E94853CEEE9F1E00E9415
:104700004539E8E6F1E00E9440390E9464390E9490
:104710004D3AEDE0F0E0AEE9B1E00E94853C0E9448
:1047200060330091EF01053011F00C94B22381E069
:104730008093020181E08093030188278093040124
:10474000A4EDB1E00E94F135E8ECF1E80E94F73504
:10475000A7E9B4E00E94F135ECE8F1E80E94F735F2
:104760000C94CB2388E08093020181E080930301C5
:10477000882780930401A4EDB1E00E94F135E8ECB4
:10478000F1E80E94F735A7E9B4E00E94F135ECE8C2
:10479000F1E80E94F73584E690E00E94673603B1A5
:1047A0004EE00423A5E0B1E00C9300910501083030
:1047B00011F00C94DD230C946C22709188017062CE
:1047C0007093880100910501023011F00C94AB2424
:1047D0000E94063580E08A93A0E9B4E08C918A9328
:1047E0008FE78A93A0E9B4E08C918A9380E08A9362
:1047F0000E943938A0E9B4E00E948835A0E9B4E00D
:104800000D911C910F3350E015071CF011F00C9422
:104810000B240C9411248FE390E0A0E9B4E08D9375
:104820009C9380E08A93A0E9B4E08C918A938FE70F
:104830008A93A0E9B4E08C918A9381E08A930E94E4
:104840003938ACE8B4E08C918A9380E08A93ACE884
:10485000B4E08C918A938FE38A9381E08A930E94DB
:1048600039380091EF01053011F40C94582480E0A0
:1048700080939204009192040F3718F011F00C9479
:104880005824A2E9B4E04C91A2E9B4E0AD90BB2475
:10489000A5EFB3E0AA0DBB1D5C9191E00E94123818
:1048A000A2E9B4E08C918F5F8C9310F40C943A24BD
:1048B0000E9460330091EF01053011F00C947B24CD
:1048C00081E08093020181E0809303018827809337
:1048D0000401A4EDB1E00E94F135E8ECF1E80E949A
:1048E000F735A7E9B4E00E94F135ECE8F1E80E9461
:1048F000F7350C94942488E08093020181E0809342
:104900000301882780930401A4EDB1E00E94F135F2
:10491000E8ECF1E80E94F735A7E9B4E00E94F13530
:10492000ECE8F1E80E94F73584E690E00E946736F3
:1049300003B14EE00423A5E0B1E00C930091050122
:10494000023011F00C94A6240C94EA237091880193
:1049500070627093880100910501063011F00C948B
:1049600072250E94063580E08A93A0E9B4E08C911C
:104970008A938FE78A93A0E9B4E08C918A9380E0D0
:104980008A930E943938A0E9B4E00E948F35A0E9EB
:10499000B4E00D911C91003050E015070CF402C0FA
:1049A0000C94D624A0E9B4E00E94A33B80E08A9353
:1049B000A0E9B4E08C918A938FE78A93A0E9B4E0F0
:1049C0008C918A9381E08A930E943938ACE8B4E0F4
:1049D0008C918A9380E08A93ACE8B4E08C918A93BE
:1049E0008FE38A9381E08A930E9439380091EF0126
:1049F000053011F40C941D2580E080939204009101
:104A000092040F3718F011F00C941D25A2E9B4E0C0
:104A10004C91A2E9B4E0AD90BB24A5EFB3E0AA0DA0
:104A2000BB1D5C9191E00E941238A2E9B4E08C9128
:104A30008F5F8C9310F40C94FF240E9460330091DC
:104A4000EF01053011F00C94402581E080930201C4
:104A500081E080930301882780930401A4EDB1E0F5
:104A60000E94F135E8ECF1E80E94F735A7E9B4E0DF
:104A70000E94F135ECE8F1E80E94F7350C945925D5
:104A800088E08093020181E080930301882780936E
:104A90000401A4EDB1E00E94F135E8ECF1E80E94D8
:104AA000F735A7E9B4E00E94F135ECE8F1E80E949F
:104AB000F73584E690E00E94673603B14EE00423A8
:104AC000A5E0B1E00C9300910501063011F00C94C3
:104AD0006D250E9406350C94B32470918801706294
:104AE000709388010C94CE190C94CE060E94662611
:104AF00081E08093EA040091EA04003818F011F094
:104B00000C94272641E050E060E070E0A8E7B1E0B7
:104B10000D911D912D913C910E94143C11F00C942B
:104B2000C525EAE8F1E00E9440390E9464390E94FC
:104B30009B392F933F934F935F93EAEEF4E0D0803D
:104B4000EE24FF2400270E9464395F914F913F912A
:104B50002F910E940C3AEDE0F0E0AEE9B1E00E9446
:104B6000853CEEE9F1E00E944539E8E6F1E00E947B
:104B700040390E9464390E944D3AEDE0F0E0AEE920
:104B8000B1E00E94853C0C940526EAEEF4E0D0806A
:104B9000EE24FF2400270E9464390E949B39E2E939
:104BA000F1E00E9440390E940C3AEDE0F0E0AAE901
:104BB000B1E00E94853CE6E9F1E00E944539EAE96E
:104BC000F1E00E9440390E944D3AEDE0F0E0AAE9A0
:104BD000B1E00E94853CEAE9F1E00E944539EAE350
:104BE000FDE70E949F3A0E94203EEDE0F0E0AAE936
:104BF000B1E00E94853CEAE9F1E00E94803DEDE0F1
:104C0000F0E0AEE9B1E00E94853C0E94FB2681E025
:104C100090E00E94673600917C00007E0760009360
:104C20007C000E94CF38AAEEB4E0AD90BB24A3EF85
:104C3000B2E0AA0CBB1CAA0DBB1D8D939C93AAEEDF
:104C4000B4E08C918F5F8C9310F40C947B250895C5
:104C5000A881B9818D919C91ADEEB4E08D939C9328
:104C60005B9881E08093EF040091EF04003118F02D
:104C700011F00C946426ADEEB4E00D911C9140E06F
:104C800050E804231523ABEEB4E00D931C93ABEE78
:104C9000B4E00D911C91003050E8150711F00C9410
:104CA00054265D9A0C9455265D985C985C9A91E028
:104CB000ADEEB4E00E94E638AFEEB4E08C918F5FC9
:104CC0008C9310F40C9434265B9A0895ACE6B1E012
:104CD0004D915D916D917C91A8E6B1E00D911D9192
:104CE0002D913C910E94143C11F00C947D26AEE86D
:104CF000B1E00E94A53B0C94FA26ACE6B1E00D9120
:104D00001D912D913C91A8E6B1E04D915D916D9181
:104D10007C910E940F3CAAE8B1E00D931D932D9366
:104D20003D93AAE8B1E00D911D912D913C9140E891
:104D300050E060E070E00E940A36AAE8B1E04D93CE
:104D40005D936D937D9342E050E060E070E0A8E7F2
:104D5000B1E00D911D912D913C910E94143C11F0F8
:104D60000C94FA26ECE6F1E00E9440390E94643986
:104D7000A2E9B1E00E949639E2E9F1E00E94863EA4
:104D8000EDE0F0E0A2E9B1E00E94853CE8E6F1E068
:104D90000E9440390E946439A6E9B1E00E94963928
:104DA000E6E9F1E00E94863EEDE0F0E0A6E9B1E040
:104DB0000E94853CE6E9F1E00E944539E2E9F1E034
:104DC0000E9440390E943E3AEDE0F0E0A2E9B1E0F5
:104DD0000E94853CEAE6FDE70E94A83AE2E9F1E09C
:104DE0000E9440390E94B639EDE0F0E0A2E9B1E05E
:104DF0000E94853C0895EEE9F1E00E940239A4EF9B
:104E0000B4E0EDE0FF270E94853CA4EFB4E00D91F3
:104E10001C914FEF5FE304231523A2EFB4E00D9341
:104E20001C9381E08093F8040091F8040E3018F090
:104E300011F00C94282791E0A4EFB4E00E94F1381F
:104E4000A8EFB4E08C918F5F8C9310F40C9414272E
:104E5000A4EFB4E00D911C914FEF5FE30423152301
:104E6000A0EFB4E00D931C93A0EFB4E00D911C9162
:104E700040E050E4040F151FA0EFB4E00D931C9325
:104E8000A2EFB4E00D911C9140E050E4040F151F17
:104E9000A2EFB4E00D931C935A924A92A4E1B1E0C0
:104EA0008D919C91D2018D939C9382E00E949838C1
:104EB0000E942826229682E00E9484355A924A92C5
:104EC000A2EFB4E08D919C91D2018D939C9382E0EE
:104ED0000E9498380E942826229682E00E948435FB
:104EE0005A924A92A0EFB4E08D919C91D2018D9399
:104EF0009C9382E00E9498380E942826229682E0A5
:104F00000E94843508950E94B43780E08093FA04AB
:104F10008BE08093F90481E08093FB040091CA0147
:104F2000033110F00C94B5274091CA010091F904A7
:104F3000041711F00C949F2781E08093FA04ABEFE3
:104F4000B4E08C918093020181E080930301AAEF89
:104F5000B4E08C9180930401E4E4FFE70E94F7350C
:104F6000ABEFB4E08C918F5F8C9380E08093FA0478
:104F7000A9EFB4E08C918F5F8C930091CA0104314A
:104F800010F00C94F2274091CA010091F904041723
:104F900011F00C94CE2781E08093FA04ABEFB4E0DB
:104FA0008C918093020181E080930301AAEFB4E029
:104FB0008C9180930401EAECF1E80E94F735ABECA8
:104FC000B1E00D91112746E050E00E949C38A0EA24
:104FD000B1E0A00FB11F0E94F135ABEFB4E08C91AE
:104FE0008F5F8C9380E08093FA04A9EFB4E08C91FA
:104FF0008F5F8C930091CA01053110F00C948528C5
:105000004091CA010091F904041711F00C940B2887
:1050100081E08093FA04E2E3F1E00E9440390E94CB
:1050200064390E949B392F933F934F935F93E8E637
:10503000F1E00E9440390E9464395F914F913F91A5
:105040002F910E94B639EDE0F0E0ABEEB1E00E94A6
:10505000853CA0E8BFE0AF93BF93EBEEF1E00E9488
:1050600040390E94763611E004E0BF91AF910E9472
:10507000C23BE0E8FFE0A4EDB1E00E94803CEBEE33
:10508000F1E00E944039EAE3FDE70E94A83A0E945D
:10509000B13A10F00C946728ABEFB4E08C91809398
:1050A000020181E080930301AAEFB4E08C91809328
:1050B0000401E6EDF1E80E94F735A4EDB1E00E94AD
:1050C000F135E0EBF1E80E94F7350C948028ABEF66
:1050D000B4E08C918093020181E080930301AAEFF8
:1050E000B4E08C9180930401EEEDF1E80E94F73575
:1050F000A4EDB1E00E94F135E0EBF1E80E94F73554
:10510000ABEFB4E08C918F5F8C9380E08093FA04D6
:10511000A9EFB4E08C918F5F8C930091CA010631A6
:1051200010F00C9418294091CA010091F904041759
:1051300011F00C949E2881E08093FA04E2E3F1E000
:105140000E9440390E9464390E949B392F933F93FB
:105150004F935F93ECE6F1E00E9440390E9464397E
:105160005F914F913F912F910E94B639EDE0F0E0B1
:10517000ABEEB1E00E94853CA0E8BFE0AF93BF93E7
:10518000EBEEF1E00E9440390E94763611E004E037
:10519000BF91AF910E94C23BE0E8FFE0A4EDB1E017
:1051A0000E94803CEBEEF1E00E944039EAE3FDE72B
:1051B0000E94A83A0E94B13A10F00C94FA28ABEF82
:1051C000B4E08C918093020181E080930301AAEF07
:1051D000B4E08C9180930401E6EEF1E80E94F7358B
:1051E000A4EDB1E00E94F135E0EBF1E80E94F73563
:1051F0000C941329ABEFB4E08C918093020181E011
:1052000080930301AAEFB4E08C9180930401EEEE49
:10521000F1E80E94F735A4EDB1E00E94F135E0EB32
:10522000F1E80E94F735ABEFB4E08C918F5F8C937F
:1052300080E08093FA04A9EFB4E08C918F5F8C93A7
:105240000091CA01073110F00C946A294091CA01FB
:105250000091F904041711F00C94312981E0809336
:10526000FA0441E050E060E070E0A8E7B1E00D91A1
:105270001D912D913C910E94143C11F00C944829F1
:10528000A2EEB1E0E6EFF1E80E94C9380C944E2995
:10529000A2EEB1E0EAEFF1E80E94C938ABEFB4E06A
:1052A0008C918093020181E080930301AAEFB4E026
:1052B0008C9180930401EEEFF1E80E94F735A2EEA5
:1052C000B1E00E94F1350E946626ABEFB4E08C910C
:1052D0008F5F8C9380E08093FA04A9EFB4E08C9107
:1052E0008F5F8C934091CA010091F904041711F06B
:1052F0000C947D2981E08093FA0441E050E060E065
:1053000070E0A4E7B1E00D911D912D913C910E94B8
:10531000143C11F00C949429A2EEB1E0ECE0F2E818
:105320000E94C9380C949A29A2EEB1E0E0E1F2E8BB
:105330000E94C938ABEFB4E08C918093020181E008
:1053400080930301AAEFB4E08C9180930401E4E11F
:10535000F2E80E94F735A2EEB1E00E94F13580E05C
:105360008093FA04ABEFB4E08C918F5F8C93A9EF3C
:10537000B4E08C918F5F8C934091CA010091F90445
:10538000041711F00C94C72981E08093FA04E2E33A
:10539000F1E00E9440390E9464390E949B392F93AA
:1053A0003F934F935F93E4E6F1E00E9440390E94FF
:1053B00064395F914F913F912F910E94B639EDE092
:1053C000F0E0ABEEB1E00E94853CA0E8BFE0AF9317
:1053D000BF93EBEEF1E00E9440390E94763611E077
:1053E00004E0BF91AF910E94C23BE0E8FFE0A4ED72
:1053F000B1E00E94803CEBEEF1E00E944039EAE32C
:10540000FDE70E94A83A0E94B13A10F00C94232ABA
:10541000ABEFB4E08C918093020181E080930301B3
:10542000AAEFB4E08C9180930401E2E2F2E80E94DA
:10543000F735A4EDB1E00E94F135E0EBF1E80E9410
:10544000F7350C943C2AABEFB4E08C9180930201C9
:1054500081E080930301AAEFB4E08C918093040172
:10546000EAE2F2E80E94F735A4EDB1E00E94F135DE
:10547000E0EBF1E80E94F73580E08093FA04A9EFB1
:10548000B4E08C918F5F8C93ABEFB4E08C918F5F25
:105490008C934091CA010091F904041711F00C9407
:1054A000542A81E08093FA040091C804013011F07D
:1054B0000C946D2AABEFB4E08C918093020181E0F3
:1054C00080930301AAEFB4E08C9180930401E2E39E
:1054D000F2E80E94F7350C94C72A023011F00C94C0
:1054E000842AABEFB4E08C918093020181E0809339
:1054F0000301AAEFB4E08C9180930401E4E4F2E8A4
:105500000E94F7350C94C72A033011F00C949B2AA3
:10551000ABEFB4E08C918093020181E080930301B2
:10552000AAEFB4E08C9180930401E6E5F2E80E94D2
:10553000F7350C94C72A043011F00C94B22AABEF63
:10554000B4E08C918093020181E080930301AAEF83
:10555000B4E08C9180930401E8E6F2E80E94F7350C
:105560000C94C72A053011F00C94C72AABEFB4E0B5
:105570008C918093020181E080930301AAEFB4E053
:105580008C9180930401EAE7F2E80E94F73580E00D
:105590008093FA04A9EFB4E08C918F5F8C93ABEF0A
:1055A000B4E08C918F5F8C930091CA01023118F0A6
:1055B00011F00C94DD2A0C94202C4091CA0100912A
:1055C000F904041711F00C94E82A81E08093FA049E
:1055D000A0E8BFE0AF93BF93ECEBF4E00E9440394A
:1055E0000E94763611E001E0BF91AF910E94C23B6C
:1055F000E0E8FFE0A4EDB1E00E94803CECEBF4E0D9
:105600000E944039EAE3FDE70E94A83A0E94B13ABD
:1056100010F00C94262BABEFB4E08C918093020138
:1056200081E080930301AAEFB4E08C9180930401A0
:10563000ECE8F2E80E94F735A4EDB1E00E94F13504
:10564000ECEBF1E80E94F7350C94182CECEBF4E04D
:105650000E944039EAE3FDE70E94A83A0E94B13A6D
:1056600081E008F480E08F93ECEBF4E00E94403995
:10567000EAE9FDE70E94A83A0E94B13A81E010F001
:1056800009F080E09F918923882311F40C94632B07
:10569000ABEFB4E08C918093020181E08093030131
:1056A000AAEFB4E08C9180930401E8E9F2E80E944B
:1056B000F735A4EDB1E00E94F135ECEBF1E80E9482
:1056C000F7350C94182CECEBF4E00E944039EEE333
:1056D000FDE70E94A83A0E94B13A81E008F480E018
:1056E0008F93ECEBF4E00E944039EEE9FDE70E9475
:1056F000A83A0E94B13A81E010F009F080E09F9151
:105700008923882311F40C94A02BABEFB4E08C9187
:105710008093020181E080930301AAEFB4E08C91B1
:1057200080930401E4EAF2E80E94F735A4EDB1E0C9
:105730000E94F135ECEBF1E80E94F7350C94182C3F
:10574000ECEBF4E00E944039E2E4FDE70E94A83A65
:105750000E94B13A81E008F480E08F93ECEBF4E032
:105760000E944039E2EAFDE70E94A83A0E94B13A5D
:1057700081E010F009F080E09F918923882311F4E3
:105780000C94DD2BABEFB4E08C918093020181E0AF
:1057900080930301AAEFB4E08C9180930401EEEAB8
:1057A000F2E80E94F735A4EDB1E00E94F135ECEB90
:1057B000F1E80E94F7350C94182CECEBF4E00E9411
:1057C0004039E6EAFDE70E94A83A0E94B13A81E03A
:1057D00008F480E08F93ECEBF4E00E944039EAEAB1
:1057E000FDE70E94A83A0E94B13A81E010F009F06A
:1057F00080E09F918923882311F40C94182CABEF3F
:10580000B4E08C918093020181E080930301AAEFC0
:10581000B4E08C9180930401E8EBF2E80E94F73544
:10582000A4EDB1E00E94F135ECEBF1E80E94F73510
:1058300080E08093FA04ABEFB4E08C918F5F8C939F
:10584000A9EFB4E08C918F5F8C930091CA01033172
:1058500018F011F00C942E2C0C94712D4091CA016B
:105860000091F904041711F00C94392C81E0809315
:10587000FA04A0E8BFE0AF93BF93E0ECF4E00E942D
:1058800040390E94763611E001E0BF91AF910E944D
:10589000C23BE0E8FFE0A4EDB1E00E94803CE0EC18
:1058A000F4E00E944039EAE3FDE70E94A83A0E9432
:1058B000B13A10F00C94772CABEFB4E08C9180935C
:1058C000020181E080930301AAEFB4E08C91809300
:1058D0000401E0ECF2E80E94F735A4EDB1E00E948B
:1058E000F135E4ECF1E80E94F7350C94692DE0EC19
:1058F000F4E00E944039EAE3FDE70E94A83A0E94E2
:10590000B13A81E008F480E08F93E0ECF4E00E948B
:105910004039EAE9FDE70E94A83A0E94B13A81E0E5
:1059200010F009F080E09F918923882311F40C94F2
:10593000B42CABEFB4E08C918093020181E08093B2
:105940000301AAEFB4E08C9180930401ECECF2E83F
:105950000E94F735A4EDB1E00E94F135E4ECF1E8E6
:105960000E94F7350C94692DE0ECF4E00E94403978
:10597000EEE3FDE70E94A83A0E94B13A81E008F404
:1059800080E08F93E0ECF4E00E944039EEE9FDE71F
:105990000E94A83A0E94B13A81E010F009F080E03C
:1059A0009F918923882311F40C94F12CABEFB4E080
:1059B0008C918093020181E080930301AAEFB4E00F
:1059C0008C9180930401E8EDF2E80E94F735A4ED94
:1059D000B1E00E94F135E4ECF1E80E94F7350C9457
:1059E000692DE0ECF4E00E944039E2E4FDE70E941A
:1059F000A83A0E94B13A81E008F480E08F93E0EC8D
:105A0000F4E00E944039E2EAFDE70E94A83A0E94D1
:105A1000B13A81E010F009F080E09F91892388235A
:105A200011F40C942E2DABEFB4E08C918093020115
:105A300081E080930301AAEFB4E08C91809304018C
:105A4000E2EEF2E80E94F735A4EDB1E00E94F135F4
:105A5000E4ECF1E80E94F7350C94692DE0ECF4E0F9
:105A60000E944039E6EAFDE70E94A83A0E94B13A56
:105A700081E008F480E08F93E0ECF4E00E9440398C
:105A8000EAEAFDE70E94A83A0E94B13A81E010F0EC
:105A900009F080E09F918923882311F40C94692DEB
:105AA000ABEFB4E08C918093020181E0809303011D
:105AB000AAEFB4E08C9180930401ECEEF2E80E942E
:105AC000F735A4EDB1E00E94F135E4ECF1E80E9475
:105AD000F73580E08093FA04ABEFB4E08C918F5FF0
:105AE0008C93A9EFB4E08C918F5F8C930091CA01E5
:105AF000043118F011F00C947F2D0C94BB2D4091C3
:105B0000CA010091F904041711F00C948A2D81E068
:105B10008093FA040091E804013011F00C94982D60
:105B2000A2EEB1E0E4EFF2E80E94C9380C949E2D99
:105B3000A2EEB1E0E8EFF2E80E94C938ABEFB4E0C2
:105B40008C918093020181E080930301AAEFB4E07D
:105B50008C9180930401EEEFF2E80E94F735A2EEFB
:105B6000B1E00E94F13580E08093FA04ABEFB4E03D
:105B70008C918F5F8C93A9EFB4E08C918F5F8C93A5
:105B80000091CA01053118F011F00C94C92D0C9444
:105B9000502E4091CA010091F904041711F00C94A1
:105BA000D42D81E08093FA040091E904013011F0D2
:105BB0000C94E82DA2EEB1E0ECE0F3E80E94C938C5
:105BC00087E68093C40080E08093C5000C94332E58
:105BD000023011F00C94FA2DA2EEB1E0E2E1F3E80C
:105BE0000E94C93883E38093C40080E08093C5009D
:105BF0000C94332E033011F00C940C2EA2EEB1E075
:105C0000E8E1F3E80E94C93889E18093C40080E0AC
:105C10008093C5000C94332E043011F00C941E2E8A
:105C2000A2EEB1E0EEE1F3E80E94C93880E1809392
:105C3000C40080E08093C5000C94332E0091E904E9
:105C4000043018F011F00C94272E0C94332EA2EE91
:105C5000B1E0E4E2F3E80E94C93888E08093C40030
:105C600080E08093C500ABEFB4E08C91809302019B
:105C700081E080930301AAEFB4E08C91809304014A
:105C8000EAE2F3E80E94F735A2EEB1E00E94F135B6
:105C900080E08093FA04ABEFB4E08C918F5F8C933B
:105CA000A9EFB4E08C918F5F8C930091CA0106310B
:105CB00018F011F00C945E2E0C947A2E4091CA01CB
:105CC0000091F904041711F00C94692E81E080937F
:105CD000FA04ABEFB4E08C918093020181E08093F1
:105CE0000301AAEFB4E08C9180930401E6E3F3E8AA
:105CF0000E94F7350E94662608950091CA010C3073
:105D000011F00C94962EABECB1E08C918F5F8C93DC
:105D10000091CB01063018F011F00C94912E0C94E8
:105D2000942E86E08093CB010C94D2300D3011F08C
:105D30000C94FF2EA8E6B1E00D911D912D913C91A0
:105D4000ABECB1E0AD90BB24AAE1B1E0AA0CBB1C66
:105D5000AA0CBB1CAA0DBB1D4D915D916D917C9150
:105D60000E940A3CA8E6B1E00D931D932D933D934C
:105D700042E050E060E070E0A4E7B1E00D911D91D9
:105D80002D913C910E94143C11F00C94DD2EA8E65C
:105D9000B1E00D911D912D913C91A4E6B1E04D91A2
:105DA0005D916D917C910E940A3CACE6B1E00D934F
:105DB0001D932D933D930C94FD2EACE6B1E04D91D7
:105DC0005D916D917C91A8E6B1E00D911D912D91B1
:105DD0003C910E94143C1CF011F00C94F12E0C9498
:105DE000FD2EACE6B1E00D911D912D913C91A8E600
:105DF000B1E00D931D932D933C930C94D2300E3053
:105E000011F00C94432FACE6B1E00D911D912D9152
:105E10003C91ABECB1E0AD90BB24AAE1B1E0AA0C9F
:105E2000BB1CAA0CBB1CAA0DBB1D4D915D916D91B5
:105E30007C910E940A3CACE6B1E00D931D932D933A
:105E40003D93ACE5B1E04D915D916D917C91ACE6F7
:105E5000B1E00D911D912D913C910E94143C1CF0DC
:105E600011F00C94352F0C94412FACE5B1E00D915D
:105E70001D912D913C91ACE6B1E00D931D932D93B6
:105E80003C930C94D2300F3011F00C94662F41E00B
:105E900050E060E070E0A8E7B1E00D911D912D9118
:105EA0003C910E94143C11F00C945E2FA8E7B1E0E5
:105EB000EEEAFDE70E949B3B0C94642FA8E7B1E05B
:105EC000EAE4FDE70E949B3B0C94D230003111F0D4
:105ED0000C94BF2F41E050E060E070E0A4E7B1E037
:105EE0000D911D912D913C910E94143C11F00C9448
:105EF000B72FA4E7B1E0EEEAFDE70E949B3BA8E6DE
:105F0000B1E00D911D912D913C91A4E6B1E04D9130
:105F10005D916D917C910E940A3CACE6B1E00D93DD
:105F20001D932D933D93ACE5B1E04D915D916D9145
:105F30007C91ACE6B1E00D911D912D913C910E94B8
:105F4000143C1CF011F00C94A72F0C94B32FACE56B
:105F5000B1E00D911D912D913C91ACE6B1E00D9316
:105F60001D932D933C930E94B4370C94BD2FA4E74E
:105F7000B1E0EAE4FDE70E949B3B0C94D230013192
:105F800011F00C942630A4E6B1E00D911D912D91F5
:105F90003C91ABECB1E0AD90BB24AAE1B1E0AA0C1E
:105FA000BB1CAA0CBB1CAA0DBB1D4D915D916D9134
:105FB0007C910E940A3CA4E6B1E00D931D932D93C1
:105FC0003D9342E050E060E070E0A4E7B1E00D9165
:105FD0001D912D913C910E94143C11F00C942430A1
:105FE000A8E6B1E00D911D912D913C91A4E6B1E0A0
:105FF0004D915D916D917C910E940A3CACE6B1E0BF
:106000000D931D932D933D93ACE5B1E04D915D91C2
:106010006D917C91ACE6B1E00D911D912D913C917B
:106020000E94143C1CF011F00C9418300C94243095
:10603000ACE5B1E00D911D912D913C91ACE6B1E044
:106040000D931D932D933C930C94D230023111F09B
:106050000C943D30A8ECB4E08C918F5F8C93009150
:10606000C804053018F011F00C9438300C943B3013
:1060700085E08093C8040C94D230033111F00C9465
:106080007330E8ECF4E0A190BB24E4EAF4E0AA0C5D
:10609000BB1CAA0CBB1CEA0DFB1D0E944539ECEB96
:1060A000F4E00E9440390E944D3AEDE0F0E0ACEBA4
:1060B000B4E00E94853CECEBF4E00E944039E2EB56
:1060C000FDE70E94A83A0E94B13A18F011F00C9432
:1060D0006B300C947130ACEBB4E0E2EBFDE70E9466
:1060E0009B3B0C94D230043111F00C94A930E8ECB5
:1060F000F4E0A190BB24E4EAF4E0AA0CBB1CAA0CD7
:10610000BB1CEA0DFB1D0E944539E0ECF4E00E9447
:1061100040390E944D3AEDE0F0E0A0ECB4E00E947E
:10612000853CE0ECF4E00E944039E2EBFDE70E94A0
:10613000A83A0E94B13A18F011F00C94A1300C94D6
:10614000A730A0ECB4E0E2EBFDE70E949B3B0C948F
:10615000D230053111F00C94BD300091E8040030CC
:1061600011F00C94B83081E08093E8040C94BB30BB
:1061700080E08093E8040C94D230063111F00C9446
:10618000D230A9EEB4E08C918F5F8C930091E9043A
:10619000053018F011F00C94CF300C94D23085E01B
:1061A0008093E90408950091CA010C3011F00C9419
:1061B000E9308091CB0181508093CB010091CB01DC
:1061C000013010F00C94E73081E08093CB010C9407
:1061D0005F330D3011F00C944E31A8E6B1E00D9113
:1061E0001D912D913C91ABECB1E0AD90BB24AAE1A7
:1061F000B1E0AA0CBB1CAA0CBB1CAA0DBB1D4D9187
:106200005D916D917C910E940F3CA8E6B1E00D93E9
:106210001D932D933D93A0E6B1E04D915D916D915D
:106220007C91A8E6B1E00D911D912D913C910E94C9
:10623000143C0CF402C00C942931A0E6B1E00D919D
:106240001D912D913C91A8E6B1E00D931D932D93E6
:106250003C9342E050E060E070E0A4E7B1E00D91D3
:106260001D912D913C910E94143C11F00C944C31E5
:10627000A8E6B1E00D911D912D913C91A4E6B1E00D
:106280004D915D916D917C910E940A3CACE6B1E02C
:106290000D931D932D933D930C945F330E3011F0AD
:1062A0000C949031ACE6B1E00D911D912D913C9193
:1062B000ABECB1E0AD90BB24AAE1B1E0AA0CBB1CF1
:1062C000AA0CBB1CAA0DBB1D4D915D916D917C91DB
:1062D0000E940F3CACE6B1E00D931D932D933D93CE
:1062E000A8E6B1E04D915D916D917C91ACE6B1E095
:1062F0000D911D912D913C910E94143C0CF402C013
:106300000C948E31A8E6B1E00D911D912D913C9138
:10631000ACE6B1E00D931D932D933C930C945F3349
:106320000F3011F00C94B33141E050E060E070E0C8
:10633000A8E7B1E00D911D912D913C910E94143C74
:1063400011F00C94AB31A8E7B1E0EEEAFDE70E9452
:106350009B3B0C94B131A8E7B1E0EAE4FDE70E9471
:106360009B3B0C945F33003111F00C940C3241E0F4
:1063700050E060E070E0A4E7B1E00D911D912D9137
:106380003C910E94143C11F00C940432A4E7B1E05B
:10639000EEEAFDE70E949B3BA8E6B1E00D911D915E
:1063A0002D913C91A4E6B1E04D915D916D917C9170
:1063B0000E940A3CACE6B1E00D931D932D933D93F2
:1063C000ACE5B1E04D915D916D917C91ACE6B1E0B1
:1063D0000D911D912D913C910E94143C1CF011F0E7
:1063E0000C94F4310C940032ACE5B1E00D911D91A8
:1063F0002D913C91ACE6B1E00D931D932D933C9310
:106400000E94B4370C940A32A4E7B1E0EAE4FDE755
:106410000E949B3B0C945F33013111F00C94A53228
:10642000ABECB1E0AD90BB24AAE1B1E0AA0CBB1C7F
:10643000AA0CBB1CAA0DBB1D4D915D916D917C9169
:10644000A4E6B1E00D911D912D913C910E94143C68
:106450000CF402C00C944232ABECB1E0AD90BB2422
:10646000AAE1B1E0AA0CBB1CAA0CBB1CAA0DBB1D67
:106470000D911D912D913C91A4E6B1E00D931D93DA
:106480002D933C93A4E6B1E00D911D912D913C918B
:10649000ABECB1E0AD90BB24AAE1B1E0AA0CBB1C0F
:1064A000AA0CBB1CAA0DBB1D4D915D916D917C91F9
:1064B0000E940F3CA4E6B1E00D931D932D933D93F4
:1064C00042E050E060E070E0A4E7B1E00D911D9182
:1064D0002D913C910E94143C11F00C94A332A8E63B
:1064E000B1E00D911D912D913C91A4E6B1E04D914B
:1064F0005D916D917C910E940A3CACE6B1E00D93F8
:106500001D932D933D93ACE5B1E04D915D916D915F
:106510007C91ACE6B1E00D911D912D913C910E94D2
:10652000143C1CF011F00C9497320C94A332ACE59F
:10653000B1E00D911D912D913C91ACE6B1E00D9330
:106540001D932D933C930C945F33023111F00C9406
:10655000B9328091C80481508093C8040091C80466
:10656000013010F00C94B73281E08093C8040C9491
:106570005F33033111F00C94F932ECEBF4E00E943C
:106580004039E8ECF4E0A190BB24E4EAF4E0AA0C82
:10659000BB1CAA0CBB1CEA0DFB1D0E9445390E94C6
:1065A000B13A18F011F00C94DD32E8EAF4E0ACEB0B
:1065B000B4E00E94853C0C94F732E8ECF4E0A19042
:1065C000BB24E4EAF4E0AA0CBB1CAA0CBB1CEA0D39
:1065D000FB1D0E944539ECEBF4E00E9440390E941B
:1065E0003E3AEDE0F0E0ACEBB4E00E94853C0C9468
:1065F0005F33043111F00C943933E0ECF4E00E9485
:106600004039E8ECF4E0A190BB24E4EAF4E0AA0C01
:10661000BB1CAA0CBB1CEA0DFB1D0E9445390E9445
:10662000B13A18F011F00C941D33ECEAF4E0A0EC50
:10663000B4E00E94853C0C943733E8ECF4E0A19080
:10664000BB24E4EAF4E0AA0CBB1CAA0CBB1CEA0DB8
:10665000FB1D0E944539E0ECF4E00E9440390E94A5
:106660003E3AEDE0F0E0A0ECB4E00E94853C0C94F2
:106670005F33053111F00C944D330091E804003084
:1066800011F00C94483381E08093E8040C944B3370
:1066900080E08093E8040C945F33063111F00C9491
:1066A0005F338091E90481508093E9040091E9040B
:1066B000013010F00C945F3381E08093E904089579
:1066C000E0E9F4E0D190E0808FEFE7FE8827F82E34
:1066D000082F0E9464390E949B39EEE2FDE70E9478
:1066E0009F3A0E943E3AEDE0F0E0A3E9B4E00E9458
:1066F000853CE2E8F4E00E944539E3E9F4E00E94D9
:1067000040390E940C3AEDE0F0E0A3E9B4E00E94C9
:10671000853CA0E8BFE0AF93BF93E3E9F4E00E94BB
:1067200040390E94763611E001E0BF91AF910E949E
:10673000C23BE0E8FFE0A7E9B4E00E94803CACE6A1
:10674000B1E00D911D912D913C91A8E6B1E04D91E4
:106750005D916D917C910E940F3CACE0B1E00D9396
:106760001D932D933D9341E050E060E070E0A8E779
:10677000B1E00D911D912D913C910E94143C11F0BE
:106780000C943D34ACE0B1E00D911D912D913C9104
:106790004FE750E060E070E00E940A36ACE0B1E004
:1067A0004D935D936D937D93ACE0B1E00D911D91A0
:1067B0002D913C91A0E1B1E00D931D932D933C935D
:1067C000ACE0B1E00D911D912D913C91ACE8B4E0AD
:1067D0004D915D9157FB1EF46FEF7FEF02C066276E
:1067E00077270E94A638ACE0B1E00D931D932D935E
:1067F0003D930091EF01053011F00C942734ACE685
:10680000B1E00D911D912D913C91ACE0B1E04D9125
:106810005D916D917C910E940F3CACE0B1E00D93D5
:106820001D932D933D9305EE13E82EE135E0ACE08A
:10683000B1E04D915D916D917C910E940F3CACE077
:10684000B1E00D931D932D933D930C943B34ACE03C
:10685000B1E00D911D912D913C91A8E6B1E04D91D3
:106860005D916D917C910E940A3CACE0B1E00D938A
:106870001D932D933D930C94CC34E8E6F1E00E94F7
:1068800040390E946439A3E9B4E00E949639E3E9F3
:10689000F4E00E94863EEDE0F0E0A3E9B4E00E945F
:1068A000853CECE6F1E00E9440390E946439ABEE91
:1068B000B1E00E949639EBEEF1E00E94863EEDE0F9
:1068C000F0E0ABEEB1E00E94853CE3E9F4E00E9429
:1068D0004539EBEEF1E00E9440390E943E3AEDE08E
:1068E000F0E0ABEEB1E00E94853CEAE6FDE70E94F5
:1068F000A83AEBEEF1E00E9440390E94B639EDE093
:10690000F0E0ABEEB1E00E94853CECE8F4E0D19021
:10691000E0808FEFE7FE8827F82E082F0E94643969
:106920000E949B39EBEEF1E00E9440390E940C3A44
:10693000EDE0F0E0ABEEB1E00E94853CEBEEF1E083
:106940000E944539E3E9F4E00E9440390E944D3A43
:10695000EDE0F0E0ABEEB1E00E94853CEBEEF1E063
:106960000E944539EAE3FDE70E949F3A0E94203EDB
:10697000EDE0F0E0ABEEB1E00E94853CEBEEF1E043
:106980000E94803DEDE0F0E00E940239ACE0B1E011
:10699000EDE0FF270E94853CE2E3F1E00E944039F0
:1069A0000E9464390E949B392F933F934F935F93CA
:1069B000ECE0F1E00E9440390E9464395F914F9110
:1069C0003F912F910E94B639EDE0F0E0ABEEB1E0DF
:1069D0000E94853CA0E8BFE0AF93BF93EBEEF1E0EF
:1069E0000E9440390E94763611E005E0BF91AF91D8
:1069F0000E94C23BE0E8FFE0A4EDB1E00E94803CD1
:106A0000709188017F7D7093880108958AE090E0FD
:106A10000E94673608950F921F922F923F924F92D5
:106A20005F927F92AF92BF920F931F932F933F93EA
:106A30004F935F936F937F938F939F93AF93BF9386
:106A4000CF93DF93EF93FF938FB78F93A2EFB1E0D4
:106A50000E9488358F918FBFFF91EF91DF91CF9189
:106A6000BF91AF919F918F917F916F915F914F9166
:106A70003F912F911F910F91BF90AF907F905F90AA
:106A80004F903F902F901F900F9018950F921F924C
:106A90002F923F924F925F927F92AF92BF920F934D
:106AA0001F932F933F934F935F936F937F938F9396
:106AB0009F93AF93BF93CF93DF93EF93FF938FB7E2
:106AC0008F93A0EFB1E00E9488358F918FBFFF9127
:106AD000EF91DF91CF91BF91AF919F918F917F9176
:106AE0006F915F914F913F912F911F910F91BF90A7
:106AF000AF907F905F904F903F902F901F900F909E
:106B00001895481A590A0895481A8827580A089566
:106B1000ED91FC91EF5FFF4FFC93EE930895ED91A3
:106B2000FC91E150F040FC93EE93089509D00E944F
:106B30009C3800FC10D0089503D01ED001F8F9CF86
:106B40000024E89457FF02C009D0689400F80BD0E5
:106B500010F80124089502D009D008955095409569
:106B60004F5F5F4F0895E89417FF089500951095C3
:106B70000F5F1F4F68940895352F242FE894452BFD
:106B800011F468940895512F402F0027112780E1B8
:106B9000440F551F001F111F021B130B416018F4F7
:106BA000020F131F4E7F8A9599F70895A0E8BFE062
:106BB0008D91882311F00CD0FBCF08950E949B3A51
:106BC000802D11F005D0FACF08958DE001D08AE034
:106BD0000090C00005FEFCCF8093C6000895A0E899
:106BE000BFE08D91882311F00FD0FBCF08950E9454
:106BF0009B3A802D11F008D0FACF089588EE93E0EB
:106C000066D03197D9F708950C94C837089500FCE1
:106C100005D0089530D005D001F8F9CF37D03FD056
:106C20000895842F952FA62FB72FE894452B462B38
:106C3000472B11F468940895402F512F622F732F22
:106C40000027112722273327F0E2440F551F661F24
:106C5000771F001F111F221F331F081B190B2A0B40
:106C60003B0B416028F4080F191F2A1F3B1F4E7F62
:106C7000FA9559F708950024E89477FF02C006D0EA
:106C8000689400F809D010F80124089512D04F5FDD
:106C90005F4F6F4F7F4F0895E89437FF0895009539
:106CA0001095209530950F5F1F4F2F4F3F4F6894E1
:106CB0000895409550956095709508953197F1F736
:106CC0000895689462F80895E89462F80895EF933F
:106CD000FF93EE27E82BE92B31F0E0EAFFE0319754
:106CE000F1F70197D1F7FF91EF9108958DE207FD3C
:106CF0008D938F2D881F802F881F8F57082F6894A2
:106D0000F7F8802F87FF15C080958395082F80E3C3
:106D10008D938EE28D93802F815228F080E38D93A6
:106D200099279C93089544270A95802F09F196D0BE
:106D30001FC0805230F09EE49D9381E48D939D931B
:106D4000EFCF4427DF92EF92FF920F938FE1801BEA
:106D500011F0082F83D089D09EE29D930F91FF9070
:106D6000EF90DF9044270395003209F4D7CF2BD062
:106D70003F93ECEFFDE638E12F2D1E2D0D2DFF2466
:106D8000EE24DD244427000F111F221FA8F42F92A8
:106D90003F920E949B3A102C0E949B3A202C0E940A
:106DA0009B3A302C0E949B3A3197410DD21CE31C38
:106DB000F01C3F902F9001C0339631963A9519F709
:106DC0003F9107D0AFCFDD0CEE1CFF1C0A95D9F721
:106DD0000895002719E058D08F93802B11F0039568
:106DE00001C08F911A95B9F7802F882309F496CFA7
:106DF0008F91805D8D930A95D9F792CF0065CD1D57
:106E000080B2E60E40597307A0ACB90350D6DC013E
:106E1000286BEE0094357700CA9A3B0065CD1D00C3
:106E2000B2E60E0059730700ACB90300D6DC0100CE
:106E30006BEE0000357700009A3B0000CD1D00008E
:106E4000E60E000073070000B9030000DC0100003B
:106E5000EE000000770000003B000000F694E7948D
:106E6000D79447950A95D1F7089500270DD08F93B1
:106E700003958F2D8E298D29842BC1F78F91805DED
:106E80008D930A95D9F74CCF1F930F93002710E2EB
:106E9000440FDD1CEE1CFF1C001F802F9AE0890BA5
:106EA00010F0082F43951A9599F7802F0F911F9195
:106EB0000895442718D01298139A159884E69927B4
:106EC0000E9467369FEF97B9129A2ED014FCFDCF1F
:106ED00002D04FEF08D08FE30FD080EC0DD080E4CC
:106EE0000BD088EB09C0403420F0109A1198405420
:106EF0000895119A10980895149801C0149AEF9368
:106F0000FF93E0E1F0E00E945E36FF91EF9188B9D7
:106F10001398159AEF93FF93E4E0F0E00E945E3639
:106F2000FF91EF9115980895149804D017FCFCCFA9
:106F30000895149A992797B99FEF98B9EF93FF9303
:106F4000E0E1F0E00E945E36FF91EF91139A159A0E
:106F5000EF93FF93E4E0F0E00E945E36FF91EF9143
:106F600016B0159897B908954427BDDF02D04FEFAA
:106F7000BADF00E080E4C0DF88EB800FBDDF10E403
:106F80008827BCDF1A95E1F70395083099F7089533
:106F9000EF93FF93509102015F9370900301E09192
:106FA0000001F09101010E949B3A202D0E949B3A22
:106FB000302D0E949B3A002D0E949B3A8052482F10
:106FC0000E94AC3CE40FF51F70920301B32E409178
:106FD0000301509102011DD00E949B3A802D5091D7
:106FE0000401552309F0809589DF509103015395E1
:106FF00050930301BA9459F750910201539550935D
:1070000002012A9509F75F9150930201FF91EF91D8
:1070100008954A955A9567DF88EB850F6DDF80E408
:10702000840F6ACF0F921F922F923F920F939F93DC
:107030004F93052F48E00E94B83C082E4F91502FE7
:10704000242E352EE8DF75DF74DF422D532DE3DF6C
:10705000802D0E94AB3B0F91002311F0182A01C034
:107060001922812D4BDF0F913F902F901F900F9091
:107070000895AA24BB24FF24EC81EA80EE1AFF08BD
:10708000FB81298033242F1A330881E0EA14FA04A3
:107090003CF42FEF3FEFE094F094E80EFA1C02C0AE
:1070A00021E033272A143A043CF46FEF7FEF209459
:1070B0003094280E3A1C02C061E0772735D02E1498
:1070C0003F0414F009F017C0CE2CDF2CCC0CDD1CD3
:1070D000022C132C000C111C9A81E91761F0E20FAD
:1070E000A00CB11CAE14BF0424F019F0F60FAC18BC
:1070F000BD081AD0F1CFC22CD32CCC0CDD1C0E2C29
:107100001F2C000C111C9981F91711F42596089574
:10711000F60FA00CB11CA214B30424F019F0E20F76
:10712000AC18BD0801D0EFCF4E2F5F2F98817ACFDA
:10713000480E8827581E08950F92B801469F800177
:10714000479F100D569F100D0F9008950F921F929C
:107150002F92C801D901489F80014A9F90014B9FFF
:10716000202C499F100D211D321D5A9F202C589F05
:10717000100D211D321D599F200D311D689F200DBE
:10718000311D699F300D789F300D2F901F900F900B
:1071900008950E949B3A0D920020D9F708957091AE
:1071A0007A00706470937A0000907A0006FCFCCF3D
:1071B00070917A00706470937A0000907A0006FCF7
:1071C000FCCF80917800909179000895903041F043
:1071D0000D911C91000F111F9A95E1F71C930E93CE
:1071E0000895903071F00D911D912D913C9136953F
:1071F0002795179507959A95D1F73C932E931E9353
:107200000E9308953DD0992711278F2D880F80E880
:10721000F82A802F881F08F41FEF41F08F57082F9E
:1072200007FD04C0003240F08FEF01C08827982F7F
:10723000D82EE82EF82E09C08FE1801B082FF69477
:10724000E794D79497950A95D1F7112351F090952B
:10725000D094E094F09481E0980F8827D81EE81E1F
:10726000F81E0F2DFE2CED2CD92E0895D094E0940D
:10727000F09491E0D90E9927E91EF91E1095089512
:10728000D190E190F1900191089521913191419136
:1072900051910895102F90E8FF0C001F0927990FB6
:1072A000F7941078652F90E8440F551F5927990FD0
:1072B0004795607800380895FF0C90E89027110FEB
:1072C0009795F794092F0895102FBD2CDE2CEF2CE5
:1072D000F02E11234AF4B094D094E094F0949FEFF0
:1072E000B91AD90AE90AF90A0EE1FF2039F4FE2C8D
:1072F000ED2CDB2CBB240850C2F76CC032F00A9591
:10730000BB0CDD1CEE1CFF1CF9CF0E948839D4CFCA
:10731000B7FE089590E8B91611F4D0FE08959FEFD6
:10732000D91AE90AF90A09F403950895DD92ED9254
:10733000FD920C930895502F2D2D3E2D4F2D612F32
:1073400008952DEC3CEC4CEC5DE366270FC098DF14
:10735000F2DFDD24EE2490E8F92E0FE307C095DF7D
:1073600005C02227332740E251E46627552351F117
:10737000002381F18FDF71F11627005850580894CF
:10738000050B18F407FD03C025C007FD23C0469573
:1073900037952795F694E794D79422D0FF202AF0CA
:1073A000DD0CEE1CFF1C015073F09D2D969548F0EE
:1073B000DD203AF4EE202AF491E0D90E9927E91E57
:1073C000F91E7ACF07C09FE7092FF92A9FEFD92E20
:1073D000E92E0895DD24EE24FF24002711270895C7
:1073E0009F929924AA24BB2488E1D216E306F406CE
:1073F00028F0D21AE30AF40A089401C08894991C70
:10740000AA1CBB1CDD0CEE1CFF1C8A9571F7D92C45
:10741000EA2CFB2C9F9008953DDFE1F25038D1F229
:107420001627005850580894051F12F418F4CBCFB3
:1074300008F0D0CF0BD0FF202AF0BB0CDD1CEE1CD7
:10744000FF1C3ACF0F5F0BF4BECF36CF9F9299242B
:10745000AA24BB24992788E1990CAA1CBB1CDD1C1B
:10746000EE1CFF1C30F4920EA31EB41ED91EE91EA2
:10747000F91E8A9589F79F90089507DF0BDF503832
:1074800029F090E869270CC00AF045D015CF5FE3DA
:1074900022273327442701C0F8DEFCDE5038B1F341
:1074A000003899F3902F951B8BF312F434D0FACF58
:1074B000983118F0222733274427983028F0232FBB
:1074C000342F44279850F9CF992329F046953795C2
:1074D00027959A95D9F7912F962742F014D0B0F6B8
:1074E000F794E794D7940F5F8BF66DCF10D051F0DF
:1074F00008F4BCDEFF2052F2DD0CEE1CFF1C015034
:10750000CBF761CF67CFD20EE31EF41E0895D21AD7
:10751000E30AF40A0895DF92EF92FF920F931F930C
:10752000D22EE32EF42E052F162F6F915F914F91DF
:107530003F912F910895C895319600200895FBDF63
:10754000D02CF9DFE02CF7DFF02CF5DF002D0895CB
:10755000F2DF202DF0DF302DEEDF402DECDF502D5F
:10756000089507FB00680EF40F7757FB50680EF480
:107570005F7707FD02C057FF05C0D216E306F40689
:10758000050708952D153E054F05500708950E94E3
:107590006436E89488278A938A931CDF11278D919B
:1075A0008032E9F31197BBD098F08D3229F4109511
:1075B00011968C91B4D060F08E3229F411968C9192
:1075C000AED008F446C022960E94613681E008954C
:1075D0008C91A5D0D8F547D01196D0F703958D9111
:1075E0009ED0E0F38E3229F48C9199D010F411964C
:1075F000FBCF853419F0853609F055C011968C9172
:107600008ED060F08D3219F08B3221F0DCCF088003
:107610000094088211968C9182D0A8F680538983B9
:1076200011968C917CD058F49981990F990F09800B
:10763000900D990F8053890F8983873220F68981B5
:10764000988199230AF48195080F2DC08E3289F60E
:1076500011968C9164D068F606D018F011960A95B0
:10766000F8CF1196C1CF4F2D3E2D2D2DDD0CEE1CE8
:10767000FF1CA8F0DD0CEE1CFF1C88F0D20EE31EF0
:10768000F41E68F0DD0CEE1CFF1C48F0805309F07E
:107690006894D80E8827E81EF81E08F00895F42E86
:1076A000E32ED22E089534D019F116F5098308E996
:1076B00021D00695882787959F2D9F77980FF92EC3
:1076C0000150000F110F07958981882379F01AF472
:1076D0008195898306C035DE89818A958983D9F7AA
:1076E00005C03FDE89818A958983D9F7229608955E
:1076F00071DEFCCF0DD041F0FF2032F00A9531F061
:10770000DD0CEE1CFF1CD2F78894089508940895B0
:1077100000240D280E280F28002A00200895803309
:1077200020F08A3310F4089408958894089591E025
:1077300005C092E003C094E001C098E0FCDE0D9229
:107740009A95E1F7089582E001C084E099279D931E
:107750008A95E9F7089591E0882321F08894991F8C
:107760008A95E9F7892F9095089599278D9193959A
:107770008823E1F7939511968C9311978E919A95A2
:10778000D1F70895EA2FFB2F00244C918D9103949B
:107790008E32E1F711248D9113948823E1F71A9426
:1077A000101640F41197202F2119239580E38D9313
:1077B0002A95E9F7113039F59927AE2FBF2FA00D83
:1077C000B91FA00FB91F8C919C93853308F421C079
:1077D00031E08E918E32E9F38D3241F0830F8A339E
:1077E00019F480E331E001C033278C93AE1789F799
:1077F000332341F0AE2FBF2FB8DF81E34D3209F4C0
:107800003196808308958827E00DF81FE00FF81F58
:1078100080830895040F151F261F371F0895041B2A
:10782000150B260B370B0895041715072607370786
:107830000895000F111F221F331F08950095109502
:10784000209530950F5F1F4F2F4F3F4F08950191A7
:1078500010810EC001911191219130810BC00191D5
:10786000108117FF05C03FEF2FEF04C000811127E3
:107870002227332737FF03C0E1DF8DE28D93CF93BB
:10788000DF93CF92DF92EF92AA24BB24CC24DD2495
:10789000EE2440E2CAE0DD2755E093E38881890FBA
:1078A00087FD9F7083FD907F891B89935A95A9F767
:1078B000C0DFAA1CBB1CCC1CDD1CEE1C4A9551F77A
:1078C000E894EFE0FF2782910ED0EB30E0F71EF056
:1078D00068948A2D0CD088278D93EF90DF90CF90FD
:1078E000DF91CF910895982F829501D0892F8F70C5
:1078F000805D26F0803309F4089568948D9308958F
:1079000081918D938823E1F7089594E081918D937F
:107910009A95E1F70895F999FECFE1BDF2BD319650
:10792000089591E001C092E07B3751F47FB7F8945D
:10793000F2DF8D9180BDFA9AF99A9A95C9F77FBFC7
:107940007727089591E001C092E0E5DFF89A80B5CD
:107950008D939A95D1F70895FF935527F8E04695B2
:1079600008F4500F57954795FA95D1F7FF91089570
:10797000FF93881BF9E0001FFA9511F4FF91089519
:10798000881F841B18F4840F8894F5CF0894F3CFD4
:10799000002711272D913D910217130710F4022F94
:1079A000132F3197B9F708950FEF1FEF2D913D91E8
:1079B0000217130710F0022F132F3197B9F708950C
:1079C0000FEF1FEF88279927442755272D913D91C9
:1079D00001960217130720F0022F132F482F592F5B
:1079E0003197A1F7089588E00FB6F8945A924A9219
:1079F000E42DF52DA42DB52D480E8827581E0FBE59
:107A000008950FB6F894499059900FBE089538DC48
:107A10000F77089535DC3EDC0395AAF087E1DD0C95
:107A2000EE1CFF1C8A9589F00A95CAF7FF205AF0D0
:107A300000240D280E280F28002039F00A95DD0CAF
:107A4000EE1CFF1CDAF70A9537CCC4CCC3CC18DC8B
:107A50000023E2F35DDE19F4B6DC0068089585E0EA
:107A6000C3DFFF0C001F04830FE70695F79456D180
:107A7000506813DD5BDC139721E438E743ED5BEBE3
:107A8000CBDC27E831ED43E15DE3D6D02EE03CE3EB
:107A900043EC5DEBD1D022E83DEA4BE25EE3CCD093
:107AA0002CEE32E846E75EEBC7D020E931EE49EA3A
:107AB0005EE3C2D020E83FEE4FEF5EEBBDD024EC9A
:107AC0003FEF4FE75FE3B8D031DC139784818F57E6
:107AD00099F02AF4D82E0FEFE02EF02E04C0D82E05
:107AE000EE24FF240027F0DB28E132E741E35FE3E7
:107AF00093DCCBDB3497D1DC84CFC2DB80E003C0E6
:107B0000BFDB802F8078882321F0DF92EF92FF92F5
:107B10000F938F93BFDB802F839512F45BDC1BC028
:107B200080958A95885E0AF415C088501AF40CD0A6
:107B3000D92210C0DD2488501AF406D0E9220AC0E8
:107B4000EE2402D0F92206C09FEF8770990F8A9524
:107B5000EAF70895B1DB8F918823D9F35F914F91B4
:107B60003F912F910F93FDDC0F9199F390F3D6D0B5
:107B7000506893CC28DC45CF83DB86E035DF058376
:107B80000F772BE33AEA48EB5FE346DCCFDB139752
:107B900041D028F4858188236AF71CDC32CF8F77A7
:107BA00084836EDB349737DFC1DB139723E632E43F
:107BB00046E357EB31DC29ED37EA4AE159E33CD0A3
:107BC00026E538E14EEA5AEB37D026E53CE84DE1B0
:107BD0005CE332D02DEC37E543E65DEB2DD02DEEA6
:107BE0003DEF45E75EE328D028E132E741E35FEB74
:107BF00023D094D052DC9FDBDD24EE24FF240481CB
:107C00008FE7080F0695F794B1DB8581881F08F48C
:107C10009FDBF7CE3FDB8827039512F48894089505
:107C200007301AF0812F08940895FF1C881F0A95C9
:107C3000E2F7812B8894089530DC27DB3497ECCB76
:107C40000F93FF92EF92EDB7FEB7DF925F934F93E2
:107C50003F93ADB7BEB72F9306D0EDB7FEB73896BA
:107C6000EDBFFEBF089588278A93FA93EA93BA93EB
:107C7000AA930E944039EA2FFB2F0E9445390E94A7
:107C80004A39503819F40038B1F13BC0003819F4C2
:107C900057FD2CC02DC00F3771F15F3761F117FF11
:107CA00011C0E881F9810E9402398827D0FA87F94A
:107CB0008C830E946439E881F9810E9445390E94D1
:107CC000B13AC9F4EA81FB810E9440390F770E94E2
:107CD000283DE881F9810E9445390E940C3A0E94B2
:107CE000BD3D8C8187FB07F9259608950FE701C0FC
:107CF0000027882702C00FE78FEFF82EE82ED82E36
:107D0000F3CF0FE380E8F82E8827F8CFB9DAA0DEAA
:107D100029ED3BE54EED5EE30C940C3A5FE340E861
:107D200033272227089500001041862301410000D7
:107D3000E040CDCCCC3D0000803F00002041000061
:107D4000C84200007A440AD7234A0100000000001C
:107D500080430024744917B7D1386F12833A00006A
:107D6000000000004040000000420000FE42ACC5A0
:107D700027370000A04082E2473E00000044000098
:107D80005C4200006442000000BF000080BF0000B1
:107D9000A0417AE51D42BD378635CDCCC7429AF960
:107DA00079449A3F1C4600401C46F34FC3470200EB
:107DB0000000804FC347203130487A0031303048CE
:107DC0007A0020316B487A0031306B487A002031DC
:107DD00030306B0020314D487A0020202020204E8A
:107DE000412D303120202020202000006369726363
:107DF00075697420616E616C797A6572000020206B
:107E0000207665722E20372E35302020202000006D
:107E1000206D61646520627920737036667265201A
:107E200000002D2D2D2D2D2D2D2D2D2D2D2D2D2DDC
:107E30002D2D0000687474703A2F2F6C782D6E65AC
:107E4000742E706C00004F4B202D207374616E6493
:107E500061726400506F6D69617220772070617388
:107E60006D696500506F6D696172202B20510000B3
:107E7000506F6D696172206D6F6379004D6F73741F
:107E8000656B2053575200004D6F6E69746F72001E
:107E90004B616C69627261636A6100004B616C697D
:107EA000627261636A61205357520000506F6D69BE
:107EB000617220637A6573746F746C2E00003020D9
:107EC000202031302020203230202020333000008C
:107ED00020202020202020202020202020202020A2
:107EE000000020465B4D487A5D2000004D46410071
:107EF00057796B6F6E616A206B6F6C656A6E6F3A53
:107F00000000312E4F646C61637A2077656A736379
:107F100069650000322E4E616369736E696A20459F
:107F20004E5445520000437A792077796B6F6E6129
:107F300063006B616C69627261636A65206D6F6377
:107F4000793F0000506F6D69617220202020202051
:107F50002020202000004B616C69627261636A61BD
:107F60002020202020200000312E4F646C61637A95
:107F7000206F64205765202000007A726F646C6F58
:107F8000206D6F637920202020200000312E446F67
:107F90006C61637A20646F205765202000002020E8
:107FA0007A726F646C6F206D6F63792020200000FF
:107FB000322E557A796A203C2D20206920202D3ED2
:107FC0000000202069207573746177206D6F632035
:107FD0006D570000332E205A616B6F6E637A204517
:107FE0004E54455200004D6F632077206D57203D61
:107FF00020004D5043006D570000202020202020FD
:1080000020202020000075572000572000006D57C9
:10801000200064426D004D5041004D5042006462AA
:108020006D005700557A796A206D6F73746B61200B
:108030005357523A0000312E506F6C61637A2057CB
:1080400079204E413032000020207A205765206D83
:108050006F73746B612020200000322E506F6C61B2
:10806000637A205765204E413032000020207A206C
:108070004D6F6E206D6F73746B6120200000332E86
:10808000446F6C61637A20646F2057792020000070
:1080900020206D6F73746B61203530206F686D2008
:1080A0000000342E4E616369736E696A20454E5438
:1080B00045520000557A796A2070727A797374613A
:1080C000776B693A0000312E5573756E207A206700
:1080D0006E69617A642000002020656C656D656EB4
:1080E00074792020202020200000312E506F6C61F8
:1080F000637A207765207A2077790000557A796A4B
:10810000206D6F73746B61205357523A2000312EEB
:108110004F646C61637A206F6420577920200000DF
:108120004B6F6E696563206B616C6962722E000033
:10813000777374617720646F20676E69617A640079
:10814000626164616E6520656C656D656E74790051
:10815000446F6C61637A20646F205779000062611C
:1081600064616E7920756B6C616400004D494E202E
:108170003D2000004D4158203D20000044796E20F4
:108180003D200000206442004D20000064420000B9
:10819000494E4600202020202020205357523D00E9
:1081A0004D696E3D0000496E643D000046723D0021
:1081B0004D487A00513D00004C783D007548000064
:1081C00043783D00704600004D00537465703A20BE
:1081D000202020202000537461723A202000537424
:1081E00061723A20000053746F703A20200053747B
:1081F0006F703A2000004C494E004C4F47005377B7
:1082000065703A202020202020202000532F53008A
:1082100044454C004D6F64653A20202020202020EA
:10822000200044656C743A20200044656C743A2048
:1082300000004C4373743A2020202020202020305E
:108240002E3100004C4373743A202020202020203F
:108250002020203100004C4373743A20202020203D
:1082600020202020313000004C4373743A2020201D
:10827000202020202031303000004C4373743A20FD
:108280002020202020203130303000004C7220206F
:108290003A202020202020004C7220203A2020204C
:1082A000202000004C7220203A20202020004C7218
:1082B00020203A20202000004C7220203A2020006C
:1082C000437220203A2020202020200043722020CA
:1082D0003A20202020200000437220203A20202035
:1082E0002000437220203A202020000043722020EA
:1082F0003A20200059657300204E6F200000436F24
:108300006D6D3A2020202020202020002020392EB2
:1083100036002031392E32002033382E34002035FB
:10832000372E36003131352E3200537065643A20D5
:1083300020202020200053415645202020202000CE
:00000001FF
